:020000040000FA
:10000000040004001FEF0FF0086A800E396E39D02B
:10001000186A196A0A9A3BEC02F0D8A01200D30FB2
:10002000D8B40A8A2D0FC60F03E20A0FF4E305D0F5
:10003000F30FF1E2060FEFE30A0F146E040E156ED4
:10004000D89018361936152EFBD7145018120806FA
:100050000FE03BEC02F0D8A01200C60F03E20A0F3B
:1000600007E3EBD7F30F04E2060F02E30A0FE5D72D
:100070000AAA04D0181E191E184A192A1850D88026
:100080001200186A196A1A6A1B6A0A9AF4D9D8A067
:100090001200D30FD8B40A8A2D0FC60FF7E20A0F49
:1000A000F5E3146E136A126A116A0A0E106E53ECAD
:1000B00004F014501024186E1150196E000ED8B0B0
:1000C000010E192612501A6E000ED8B0010E1A2613
:1000D00013501B6E000ED8B0010E1B26080607E059
:1000E000CAD9D8A01200C60F02E20A0FDAE20AAAA1
:1000F0000BD0181E191E1A1E1B1E182AD8B4192A36
:10010000D8B41A2AD8B41B2A1850D8801200086A0A
:10011000186E196A00960850D8B40086040E076E4F
:10012000193805D8195003D8183801D818500F0BB2
:10013000F60FD8B0070F0A0F28D0086A186E196A90
:1001400018BE196832D803D0086A186E196A00966A
:100150000850D8B40086050E076E270E156E100ED7
:100160000CD8030E156EE80E08D8156A640E05D873
:10017000156A0A0E02D8185008D0146E1950116E64
:100180001850106E01EC04F01050106E074E0096DF
:10019000085003E0075CD8B007D01050D8A40096F0
:1001A00000B602D0300F59D1120019AE120018500B
:1001B0001910D8B41200181E191E184A192A2D0E2B
:1001C0004CD13B6E24AE02D02D0E47D9263E04D032
:1001D000253E02D0244A242A316A326A336A346ABC
:1001E000248E6A0E2326D8902432253226323432C9
:1001F000333232323132233EF6D72650235C262664
:10020000235E2550245C2526245E086A39D82E0EEC
:1002100024D93C6AD8903134266E3234256E33347A
:10022000246E3434236E3C36D89026362536243658
:1002300023363C36315026263250D8B0323C252663
:100240003350D8B0333C24263450D8B0343C232625
:10025000D8B03C3ED89026362536243623363C3658
:100260003C50300FFAD826C031F025C032F024C0FF
:1002700033F023C034F03B2ECCD7D890120028D8CE
:100280000096085003E100860A0E086E26C013F09F
:1002900025C012F024C011F023C010F0076A1B6AB9
:1002A0001A6A196A0A0E186ED3EC03F0072A07506F
:1002B000085CD8A4F4D71850D8A4009600A602D0A1
:1002C000082C03D01850300FC8D8082EDFD71200E2
:1002D00026AE1200D880000E2356245625562656E8
:1002E0002D0EBBD005C010F006C011F0010E146E2B
:1002F000156AEA6802C0E9FF04002AD8D8A015D020
:10030000142EFAD7FF0E1526D8B0F6D71026D8A08F
:100310001126D8A01200320E146E156AEDD7EA68C5
:1003200002C0E9FF040014D8FDE254D81E6A080E8A
:10033000156E51D80DD8D8B01E3E1432152EF9D7EF
:1003400021AA1E6A21BA149E46D8D88014501200E1
:10035000120EE9260950EF1202C0E9FFEF1421BC8A
:100360000918FF0F12001C6EEA68E2680250E96E7D
:10037000120FE16E800E0A16080E1D6ED890D8B0CE
:100380000A3E11D81C321D2EFAD7040021BA0A30B9
:100390000AD800D000D000D0D88005D80650156EFD
:1003A000055062D9120021AE0BD0EF50091021ACDC
:1003B0000918EF6EE7500910D8A00918E76E0BD0A6
:1003C000EF500910D8A0091821BC0918EF6E091CBC
:1003D000E71601D00A8C21501F0BFF0F116E205021
:1003E000F70FD8B0112A0AAC4CD10A9C106E020E3D
:1003F000A5EC04F046D171B27198718802C010F07A
:1004000009C011F0146A156A040000D00400A4BAEF
:1004100014D0E8681426152210221122D8A0120048
:100420001448153CF1D73D0E146E156AEFD771B222
:10043000719871880400A4AAFED77450D880120065
:10044000A66AA68E0900F55002E002D8FBD712007A
:100450000400A4A8FED7736E120001BA84D701A2CB
:1004600002D001B038D001A205D001B003D001B252
:10047000EE6E1200EDD73950080ABDE03950090A76
:10048000D6E03950030AD8B42DD73950050AD8B46C
:1004900046D7D88039BEEE501200008800A80098D8
:1004A00000BA03D0008A35D829E20094080E156EF0
:1004B00040D81436152EFCD700B407D000B801D0B0
:1004C0004AD845D841D800B819D843D8D890145044
:1004D0001CD0008800A8009800BC05D0FE0B0A6E56
:1004E000008CD89012D000BE05D01C6E008E11D8A2
:1004F00005E21C5012D802E200A807D02CD827D859
:10050000009C009E009A009424D81E80D8A01E90C3
:10051000120017D80A5000BA0109146E080E156EA1
:10052000143617D801E217D812D80ED8152EF8D7DE
:1005300010D80DD800D00400D89081BCD88004D841
:10054000120007D804D807D8819E939E06D0938EB8
:1005500004D0938C02D08A9C939C1200AA6AA96E44
:10056000A66AA680A850A94AAA2A1200AA6AA86E5A
:10057000A66AA684550EA76EAA0EA76EA6820400D0
:10058000A6B2FED7A694A94AAA2A1200E836E836EF
:10059000FC0B0109C2128009C216C050F80B0309F6
:1005A000C06E640E6DD8C2820400C2B2FED7C4CF42
:1005B00024F0C350236E1200080E1C6E1D6EEA68F4
:1005C00003C0E9FF04500AB4C4D90AA4C4D9E2683C
:1005D00003C0E1FFEA6802C0E9FF0950E988E92A9F
:1005E000EC1202C0E9FF106A116A1C50D8B4120064
:1005F0000AB234D8EF500914FF0F103611360AA290
:100600002DD81C2EF5D71D500AB08ED110501200D7
:10061000080E1C6EEA6803C0E9FF04500AB499D9B9
:100620000AA499D9E26803C0E1FFEA6802C0E9FFC1
:10063000091CE988E92AEC161C50D8B412000AB04B
:1006400073D902C0E9FF11321032EF500910D8A05F
:100650000918EF6E03D81C2EF6D712000450E71AC3
:100660000400E71A1200156A146EFF0E14261522F4
:1006700000D0D8A01200030E116EDE0E02D8F5D7FE
:10068000116AE90F106EFC0E05E304000400102649
:10069000FDE2040010261106F9E210B000D010A20D
:1006A00002D000D0040012000009D8B412001E6E5F
:1006B00010C0E9FF11C0EAFF116A106A1EBE07D020
:1006C000EE50106E1EA21200EF50116E120004D8F0
:1006D000EF14D8A4102A1200010E1EB0E8441EB276
:1006E000E8441EB2E8441EB4E838120013501B1848
:1006F000800BF46E13AE06D0D880000E1056115643
:10070000125613561BAE06D0D880000E1856195636
:100710001A561B56146A156A166A176A2D6A2E6ACB
:100720002F6A306A1B501A101910181023E0200E7F
:10073000F36ED89010361136123613362D362E360B
:100740002F36303618502D5C19502E581A502F580D
:100750001B50305809E318502D5E19502E5A1A506C
:100760002F5A1B50305AD880143615361636173685
:10077000F32EDFD7F4AE06D0D880000E14561556EF
:100780001656175614C010F015C011F016C012F00E
:1007900017C013F02DC018F02EC019F02FC01AF09A
:1007A00030C01BF012002D6A2E6A2F6A306A210EAB
:1007B000166E15D02D362E362F36303618502D5C4D
:1007C00019502E581A502F581B50305808E3306ECD
:1007D00018502D5E19502E5A1A502F5AD8801036A4
:1007E000113612361336162EE5D730C01BF02FC047
:1007F0001AF02EC019F02D50186E1200116A156AE9
:10080000146E196A186A100EF36E11341836193600
:100810001450185C1550195805E31450185E155003
:10082000195AD88010361136F32EEFD71050120017
:100830001F501918800BF46E1FAE05D01E1E1F1E10
:100840001E2AD8B41F2A19AE05D0181E191E182A40
:10085000D8B4192A146A106A116A156A195002E18B
:10086000185018E0100EF36ED8901E361F3614364E
:1008700015361950155C02E11850145C07E3185046
:10088000145ED8A015061950155ED88010361136A2
:10089000F32EEAD7F4AE05D0101E111E102AD8B4DC
:1008A000112A1050120013C030F012C02FF011C0E6
:1008B0002EF010C02DF02F501802F3CF12F0F4CF0D
:1008C00013F02E501902F3501226F45013222D501B
:1008D0001A02F3501226F450132230501802F3502B
:1008E00013262F501902F35013262E501A02F350DC
:1008F00013262D501B02F35013262D501802F3CF50
:1009000010F0F4CF11F02E501802F3501126F450CD
:100910001222000E13222D501902F3501126F4500A
:100920001222000E13221200146A156A04D011322A
:10093000103214361536FF0FFAE215C011F01450BC
:10094000106E1200D89011321032FF0FFBE21050DF
:100950001200EF1203D0FF0AEF1601D0FF0AE98858
:10096000E92AEC161200A66AA68E0900F55002E0EC
:10097000EE6EFBD71200A66AA68EEE500900F55C5B
:1009800002E1F566FAD712003DC01EF03D8C0ED88C
:10099000D90E386E5B0E376E5E0E366E7D0E356E7E
:1009A00094EC07F01EAC3D9C3450120032BE09D1CD
:1009B0003152D8B406D13DC01CF03D8C7E0E315C66
:1009C0001D6E7E0E316E386A376A366A7F0E356E5E
:1009D000F30E345C040ED8A0050E335C350ED8A09F
:1009E000360E325C02E3AAD903D0312AA7D91D06FC
:1009F00034C010F033C011F032C012F031C013F027
:100A0000710E386E5F0E376E550E366E800E356E77
:100A100097D910C038F011C037F012C036F013C0AB
:100A200035F094EC07F0C60E386EF50E376E1F0EDB
:100A3000366E800E356E84D934C014F033C015F094
:100A400032C016F031C017F010C034F011C033F0CE
:100A500012C032F013C031F08A0E386E120E376EAB
:100A6000790E366E7D0E356E94EC07F0F60E386E0C
:100A7000460E376E550E366E7E0E356E61D914C039
:100A800038F015C037F016C036F017C035F0E6D98B
:100A900034C014F033C015F032C016F031C017F076
:100AA0001350316E356E1250326E366E1150336EF9
:100AB000376E1050346E386E94EC07F034C023F06B
:100AC00033C024F032C025F031C026F014C038F015
:100AD00015C037F016C036F017C035F094EC07F0AB
:100AE00010C038F011C037F012C036F013C035F026
:100AF00094EC07F023C038F024C037F025C036F05E
:100B000026C035F03566350619D910C038F011C049
:100B100037F012C036F013C035F012D91D5252E032
:100B200034C023F033C024F032C025F031C026F0A9
:100B30001DC031F0000E31BEFF0E326E336E346ECA
:100B400041EC08F034C010F033C011F032C012F0A4
:100B500031C013F0830E386E800E376EDE0E366EA7
:100B6000720E356EE1D923C038F024C037F025C0AD
:100B700036F026C035F0E4D834C023F033C024F07A
:100B800032C025F031C026F010C034F011C033F06F
:100B900012C032F013C031F0386A800E376E310E59
:100BA000366E7E0E356EC0D923C038F024C037F0C3
:100BB00025C036F026C035F0C3D81CBC03D03D9C00
:100BC00001D03D8A34501200365032183F6E3FBE7D
:100BD00030D036BE17D03550315CD8A0000CD8A428
:100BE000010C3650325CD8A0000CD8A4010C375050
:100BF000335CD8A0000CD8A4010C3850345CD8A0C9
:100C0000000C010C3150355CD8A0000CD8A4010CAC
:100C10003250365CD8A0000CD8A4010C3350375C9D
:100C2000D8A0000CD8A4010C3450385CD8A0000C1B
:100C3000010C32AE010C000C365032183F6E3FBE34
:100C400034D036BE19D03550315CD8A0000CD8A4B1
:100C5000010C3650325CD8A0000CD8A4010C3750DF
:100C6000335CD8A0000CD8A4010C3850345CD8A058
:100C7000000CD8A4010C000C3150355CD8A0000C3D
:100C8000D8A4010C3250365CD8A0000CD8A4010CBA
:100C90003350375CD8A0000CD8A4010C3450385C19
:100CA000D8A0000CD8A4010C000C32AE010C000C32
:100CB000325036183F6E3FBE34D032BE19D031505C
:100CC000355CD8A0000CD8A4010C3250365CD8A0FA
:100CD000000CD8A4010C3350375CD8A0000CD8A469
:100CE000010C3450385CD8A0000CD8A4010C000CC6
:100CF0003550315CD8A0000CD8A4010C3650325CC1
:100D0000D8A0000CD8A4010C3750335CD8A0000C3C
:100D1000D8A4010C3850345CD8A0000CD8A4010C25
:100D2000000C36AE010C000C386A376A7E0E356E48
:100D3000800E32AE000E366E03D844D1800E361AC5
:100D40003550315C3C6E11E23C6C315035C031F0B5
:100D5000356E325036C032F0366E335037C033F015
:100D6000376E345038C034F0386E1A0E3C6074D090
:100D7000355272E03B6A32503E6E3618406E328E0B
:100D8000368E080E3C5E08E338C03BF037C038F0C2
:100D900036C037F0366AF5D73C2607E0D8903632B1
:100DA000373238323B323C2EF9D740AE33D0385050
:100DB000345E3750335A3650325A07E2D880000E2C
:100DC000345633563256800E3E1A3B6C04E03406DD
:100DD000000E335A325A040E3C6E32660DD033C0C8
:100DE00032F034C033F03BC034F03B6A080E315E61
:100DF00029E33C2EF2D726D032BE08D0D8903B361D
:100E0000343633363236312EF7D71CD03BAE22D0B3
:100E10003B6A0FD0385034263750332236503222B6
:100E200006E33232333234323B32314A0DD03BAEFC
:100E300011D0343E0FD0333E0DD0323E0BD0D8808F
:100E40003490EFD7316A02D03D823168346A336A18
:100E5000800E326E3EAE329E3450120032502F6EF3
:100E60003618406E355051E0315252E0315E7F0EFF
:100E700003E2312603E24BD031264CE234C02DF0A0
:100E800033C02EF02F8E368E180E3E6E346A336AC3
:100E9000326A0BD038502D5C37502E5811E32E6E2D
:100EA0002F6A38502D5E0BD004E236502F5CF2E0F2
:100EB00007E338502D5E37502E5A36502F5AD880BF
:100EC0003436333632362D362E362F363E2EECD78C
:100ED00032BE07D031521BE0403231063E2A403646
:100EE000E3D707E238502D5E37502E5A36502F5A2E
:100EF00017E3343E15D0333E13D0323E11D0323298
:100F000033323432313E0CD005D03D8604D03D849E
:100F1000316A02D03D823168346A336A800E326EA3
:100F200040AE329E3450120032502F6E3618406E52
:100F30003150D8A435503AE031267E0E03E3315EBD
:100F400003E336D0315E31E334C02DF033C02EF0F0
:100F50002F8E368E346A336A326A180E3E6E2F3206
:100F60002E322D3206E33850342637503322365095
:100F700032223232333234323E2EF1D732BE07D0F3
:100F8000343633363236315210E031062F3416E320
:100F9000343E14D0333E12D0323E10D0D88032329C
:100FA00033323432313E0AD003D03D84316A02D02C
:100FB0003D823168346A336A800E326E40AE329EB2
:100FC0003450120031C03EF0325034C032F0346E32
:100FD00034363E3234323D6A34363E3602E33D84A6
:100FE0003D7E06E13D803E6A346A336A326A0BD048
:100FF0003E2803E0D880343206D0D890343202E163
:101000003D8201D03D863DB604D03DA20FD03DB417
:1010100007D07F0E346EFF0E336E326E316E23D0EA
:10102000800E346E01D0346A000EF6D73DB0FBD787
:10103000316A9F0E3E60EBD77E0E3E64F4D79E0E63
:101040003E5C07E0D89034323332323231323E2ABD
:10105000F6D73DA408D0D880000E3156325633560C
:10106000345634AEE0D731501200000E32BEFF0EBF
:10107000336E346E06D0316E326A336A346A409E03
:101080000AD0409E34AE07D0D880000E315632567A
:1010900033563456408E960E3E6E345209E0080E9A
:1010A0003E2632C031F033C032F034C033F011D0BC
:1010B00033520FE1080E3E5E325007E1080E3E5EED
:1010C000315002E1345010D0316A336E31C032F009
:1010D000316A33BE06D0D8903136323633363E06CA
:1010E000F8D740AE339E3E5031C034F0316E3350AD
:1010F00032C033F0326E120024505542582C343036
:101100002C474C4C2C302C302C302C302A354300C2
:1011100024505542582C34302C5A44412C302C3019
:101120002C302C302A34340024505542582C343082
:101130002C4753562C302C302C302C302A3539008B
:1011400024505542582C34302C4753412C302C30ED
:101150002C302C302A34450024505542582C343041
:101160002C524D432C302C302C302C302A3437006C
:1011700024505542582C34302C4747412C312C30C8
:101180002C302C302A35420024504D544B3331340E
:101190002C302C302C302C312C302C302C302C306E
:1011A0002C302C302C302C302C302C302C302C305F
:1011B0002C302C302C302A32390024505542582CF7
:1011C00034302C5654472C302C302C302C302A35CF
:1011D000450024504D544B3331342C302C302C31BD
:1011E0002C312C302C302C302C302C302C302C301E
:1011F0002C302C302C302C302C302C302C302C300F
:101200002A32380024505542582C34302C5654473A
:101210002C312C302C302C302A35460024504D54A3
:101220004B3136312C302A32380024504D544B315A
:1012300030322A3331002447504747412C30303276
:101240003135332E3030302C343831352E3930387A
:10125000302C4E2C30313934392E323132302C454D
:101260002C312C31302C312E322C3231372E302C87
:101270004D2C2D33342E322C4D2C2C303030302A46
:10128000354500002447505654472C3330392E360C
:10129000322C542C202C4D2C302E31332C4E2C3013
:1012A0002E322C4B2C412A32330020202020475054
:1012B0005320434F4D4D554E49434154494F4E20C5
:1012C0004552524F5220202000002020202047501D
:1012D0005320435243204552524F522020200000B9
:1012E00042414C4C4F4F4E205041594C4F414420AD
:1012F00056200000204259204F4D3342430054797C
:1013000070652048454C5020666F7220496E666FAC
:1013100000004357494400004357430043574341AB
:101320004C4C000043574C0043574C4F43004C4F2C
:101330004341544F52004C4F4331300043414C4CD9
:101340000000465251004652455155454E43590002
:1013500044455600444556494154494F4E00424188
:1013600055440000535045454400444249545300FD
:10137000534249545300504F55540000504F574565
:101380005200494453500000435753500000534FFC
:101390004C41520055534F4C000049534F4C0000F4
:1013A00054454D500000494E54454D50000045589D
:1013B00054454D5000005052455353005052455330
:1013C000535552450000435742415400435754453A
:1013D0004D500000434F5552534500004241545672
:1013E000000053555056000053454E5400004449E8
:1013F00053500000524546005443584F00004F469A
:1014000046534554000048454C5000004441544167
:101410000000534C4545500054455354000054556A
:101420004E450000534552475053000043414C493C
:101430004252415445005345545000004E4F4750CE
:10144000530055424C4F5800564552004558495498
:101450000000436F6D6D616E64206973206E6F7460
:101460002076616C6964000055202D204652512081
:1014700055702C2044202D2046525120446F776E09
:101480002C2045202D2045786974000055424C4F92
:1014900058200000534F4C415263656C6C20000093
:1014A00054454D5065726174757265200000494E57
:1014B0007465726E616C54454D50657261747572DD
:1014C0006520000045587465726E616C54454D503E
:1014D00065726174757265200000737065656420C3
:1014E0002620434F555253452000424154566F6CBD
:1014F000746167652000535550706C79566F6C7439
:10150000616765200000536F6C6172566F6C746187
:1015100067652000536F6C617243757272656E74FB
:10152000200053454E54656E636520004357424189
:1015300054200000435754454D5020004C4F434128
:10154000544F522000004C4F43313020000043578D
:101550004C4F432000005052455353757265200094
:10156000534C45455020000043414C4C3A2000006C
:10157000435743414C4C3A20000046524551554593
:101580004E43593A2000444556494154494F4E3A3A
:10159000200053504545443A2000444154412042E4
:1015A0004954533A200053544F5020424954533A1F
:1015B0002000504F574552204F55543A2000435772
:1015C00049442073706565643A2000004D4F4445DE
:1015D0004D204F46465345543A200000584F204670
:1015E00052455155454E43593A2000005345524704
:1015F00050532000343830302042640039363030C7
:1016000020426400313932303020426400004F53B0
:101610004354554E453A200056455253494F4E3A91
:10162000204243504C20762E0000564261743A20EE
:10163000000054656D703A200000436F6D6D616E5F
:101640006473202877697468206578616D706C65B3
:10165000293A2000444953502020202D20646973EA
:10166000706C617920616C6C20736574696E67734E
:10167000000043414C4C2020202D206964656E748D
:10168000696669657220666F72207061796C6F613E
:101690006400435743414C4C202D2043572069643C
:1016A000656E74696669657200004652512020209B
:1016B000202D206672657175656E637920696E20D4
:1016C000487A0000504F574552206F7220504F55B6
:1016D00054202D206F757470757420706F7765724B
:1016E00020696E206D570000524546202020202D95
:1016F00020584F206F72205443584F2066726571F6
:1017000075656E637920696E20487A20286D696E50
:101710002E2031303030303030302C206D61782E3A
:10172000203333303030303030005443584F202095
:10173000202D20594553203D205443584F2C204EF6
:101740004F203D20584F00004F4646534554202D12
:10175000206D6F64656D206672657175656E637965
:10176000206F666673657420696E20487A20286D44
:1017700061782E202B2D3330303030290000444545
:1017800056202020202D20646576696174696F6E73
:1017900020696E20487A0000424155442020202DC7
:1017A00020626175647261746520666F72205254A4
:1017B0005459207472616E736D697474696E670038
:1017C000444249545320202D206E756D626572206D
:1017D0006F66206461746162697473005342495496
:1017E0005320202D206E756D626572206F66207308
:1017F000746F706269747320312E35203D2031354D
:10180000000049445350206F722043575350202DFD
:10181000207370656564206F662043572069646596
:101820006E74696669657220696E2057504D0000BC
:10183000435749442020202D2073656E6420435770
:10184000206964656E746966696572205945532024
:101850006F72204E4F00435742415420202D207379
:10186000656E642062617465727920766F6C746154
:10187000676520696E204357202D20594553206FFE
:1018800072204E4F0000435754454D50202D207379
:10189000656E642074656D70657261747572652023
:1018A000696E204357202D20594553206F72204EDA
:1018B0004F0043574C202020202D2073656E64205C
:1018C000515241206C6F632E20616E6420616C74F4
:1018D000697475646520696E204357202D20594531
:1018E00053206F72204E4F00434F55525345202DC9
:1018F0002073656E6420636F7572736520616E641A
:10190000207370656564202D20594553206F722027
:101910004E4F0000424154562020202D2073656E0A
:10192000642062617465727920766F6C746167659A
:10193000202D20594553206F72204E4F00005355E3
:1019400050562020202D2073656E642073757070B2
:101950006C7920766F6C74616765202D2059455332
:10196000206F72204E4F0000505245535320202DBF
:101970002070726573737572652073656E736F7214
:10198000206D6F756E746564202D20594553206F4E
:1019900072204E4F20616E642073656E64207072F9
:1019A0006573737572650000534F4C415220202DB2
:1019B00020736F6C617263656C6C206D6F756E74F3
:1019C000656420594553206F72204E4F00005553D7
:1019D0004F4C2020202D2073656E6420736F6C6146
:1019E0007220766F6C74616765202D2059455320F5
:1019F0006F72204E4F0049534F4C2020202D2073F2
:101A0000656E6420736F6C61722063757272656EAF
:101A10007420594553206F72204E4F0055424C4F51
:101A20005820202D204F4E203D2055424C4F58200D
:101A30004F4646203D205155454354454C005445A2
:101A40004D502020202D2073656E6420696E626FDA
:101A5000782074656D7065726174757265202D20D3
:101A6000594553206F72204E4F00494E54454D50FA
:101A7000202D2073656E6420726164696F636869EC
:101A8000702074656D7065726174757265202D20AB
:101A9000594553206F72204E4F00455854454D50C4
:101AA000202D2073656E642065787465726E616C9C
:101AB0002074656D7065726174757265202D205992
:101AC0004553206F72204E4F00004C4F4341544FFE
:101AD000522D2073656E6420515241206C6F6361FA
:101AE000746F72202D20594553206F72204E4F0085
:101AF0004C4F43313020202D2073656E64203130EF
:101B000020636861722E206F6620515241206C6FF5
:101B1000632E204F4E203D2031302C204F46462052
:101B20003D20362063686172616B746572730000DA
:101B300053454E542020202D2073656E64204F4E57
:101B4000203D2073656E74656E6365202F204F46BF
:101B500046203D2076697369626C65207361746507
:101B60006C6974657300534C45455020202D2073DB
:101B700077697463682074686520475053207265E4
:101B800063656976657220746F2068796265726E2C
:101B9000617465206D6F6465202D20594553206F59
:101BA00072204E4F0000534552475053202D206263
:101BB00061756472617465206F66204750532072AE
:101BC00065636569766572202834383030206F721D
:101BD0002039363030206F722031393230302900D0
:101BE00054554E452020202D20736574207468655F
:101BF000205874616C206672657175656E6379003A
:101C0000444154412020202D206964656E7469662A
:101C100069636174696F6E206F6620726164696FB9
:101C2000206368697000564552202020202D2073C3
:101C30006F6674776172652076657273696F6E0086
:101C4000455849542020202D20656E64206F662061
:101C5000636F6D6D616E6420696E7465727072651C
:101C60007465720043686970205265766973696FA4
:101C70006E3A2000506172743A205369000050613E
:101C80007274204275696C643A20307800004465B3
:101C9000736372697074696F6E2049643A2030789A
:101CA0000000437573746F6D65722049643A20308B
:101CB0007800524F4D2049643A20307800004E4F52
:101CC000542056495349424C4520534154454C49B0
:101CD000544553004C6F772063757272656E743D86
:101CE00020002020486967682063757272656E74F1
:101CF0003D20000053617665643A20004E6F7420E9
:101D00007361766564202D2041637475616C207663
:101D1000616C75653A2000004E6F20677073206417
:101D20006174612072656365697665640000525371
:101D300053493A20000008000000090000000A0092
:101D400000000B0000000C0000000D0000000E0061
:101D50000000100000001200000014000000170036
:101D600000001A0000001E000000220000002700F2
:101D700000002D00000036000000460000005E005C
:101D800000007F0000007F0000007F0000000800CE
:101D90000000090000000A0000000B0000000C0019
:101DA00000000D0000000E000000100000001200F6
:101DB000000014000000170000001A0000001E00C0
:101DC000000022000000270000002D000000360067
:101DD0000000460000005E0000007F0000007F0061
:101DE00000007F00000008000000090000000A0059
:101DF00000000B0000000C0000000D0000000E00B1
:101E00000000100000001200000014000000170085
:101E100000001A0000001E00000022000000270041
:101E200000002D00000036000000460000005E00AB
:101E300000007F0000007F0000007F000000400ED7
:101E40003D6E006A060E756E200E726E900E716EFB
:101E50000001AB0E926E9A0E936E0F0E946ED20E20
:101E6000D36ED26A9B6A796A786AF26AF16AF06A1A
:101E7000816A010EC26E080EC16EAB0EC06E0B0EF3
:101E80000F01386F396B080E3A6FE00E426F416FE9
:101E9000100E406F040E9D6EA06A9F6EA26A030E24
:101EA000D56ECD6ABA6AB16A516B4E6B4A6BC66A1F
:101EB0006C6AAB9E708672987284766A670E756ED5
:101EC000900E716E03012A992A97296B1D0E040149
:101ED0001F6F4C0E1E6F949A8B8A5A0E41620AD065
:101EE0005A0E426207D05A0E436204D044505A0A36
:101EF000000102E0000E01D0010E3A6E000E030157
:101F00003EB1010E3A1600012BE0270E156E100EA1
:101F100034EC03F0FBEC36F09A0E346E990E336E0F
:101F2000190E326E7F0E316E00C338F0FFC237F0EB
:101F3000FEC236F0FDC235F0E4EC05F00108E5E044
:101F40000201C06B970E0201C05D000109E2070E9D
:101F5000156ED00E34EC03F00201C02B0001F2E349
:101F60005A0E446E436E426E416E8DEC31F03AEC87
:101F70001FF072EC1DF0D1EF1FF003013E51000184
:101F8000E8A602D0C2EC43F0719E03013D3500018A
:101F9000D8A02AD2800E026E400E096E216A40C37C
:101FA00020F0066A056A200E016EB50EB3EC01F052
:101FB000620EB3EC01F0060EB3EC01F03B0EB3EC95
:101FC00001F02C0EB3EC01F0000EB3EC01F0010EA9
:101FD000B3EC01F0060EB3EC01F0000EB3EC01F02F
:101FE000000EB3EC01F0200EB3EC01F0900EB3EC58
:101FF00001F0000EB3EC01F0000EB3EC01F0000EA6
:10200000B3EC01F0000EB3EC01F0000EB3EC01F004
:10201000000EB3EC01F0000EB3EC01F0800E026E86
:10202000400E096E216A40C320F0066A056A200E40
:10203000016E000EB3EC01F0000EB3EC01F0000EE7
:10204000B3EC01F0000EB3EC01F0000EB3EC01F0C4
:10205000000EB3EC01F0000EB3EC01F0000EB3EC97
:1020600001F0000EB3EC01F0000EB3EC01F0000E35
:10207000B3EC01F02C0EB3EC01F0010EB3EC01F067
:10208000000EB3EC01F0000EB3EC01F04F0EB3EC18
:1020900001F0C10EB3EC01F0030EB3EC01F0000E41
:1020A000B3EC01F0800E026E400E096E216A40C34F
:1020B00020F0066A056A200E016E860EB3EC01F070
:1020C000020EB3EC01F0000EB3EC01F0000EB3EC25
:1020D00001F0FE0EB3EC01F0000EB3EC01F0000EC7
:1020E000B3EC01F0000EB3EC01F0640EB3EC01F0C0
:1020F000400EB3EC01F0010EB3EC01F0000EB3ECB6
:1021000001F08F0EB3EC01F0870EB3EC01F0640E1A
:1021100033EC03F0800E026E400E096E216A40C35C
:1021200020F0066A056A200E016EB50EB3EC01F0D0
:10213000620EB3EC01F0060EB3EC01F0160EB3EC38
:1021400001F0080EB3EC01F0000EB3EC01F0000E4C
:10215000B3EC01F0030EB3EC01F0030EB3EC01F0AD
:10216000000EB3EC01F0510EB3EC01F0A20EB3EC93
:1021700001F0060EB3EC01F0000EB3EC01F0230EFB
:10218000B3EC01F0E70EB3EC01F0640E33EC03F0B6
:10219000800E026E400E096E216A40C320F0066A6E
:1021A000056A200E016EB50EB3EC01F0620EB3ECC1
:1021B00001F0060EB3EC01F0110EB3EC01F0020ECB
:1021C000B3EC01F0000EB3EC01F0080EB3EC01F03B
:1021D000010EB3EC01F0220EB3EC01F0920EB3EC61
:1021E00001F0B50EB3EC01F0620EB3EC01F0060E97
:1021F000B3EC01F0090EB3EC01F00D0EB3EC01F0FD
:10220000000EB3EC01F0000EB3EC01F0000EB3ECE5
:1022100001F0000EB3EC01F0000EB3EC01F0FF0E84
:10222000B3EC01F0FF0EB3EC01F0000EB3EC01F0E3
:10223000000EB3EC01F0000EB3EC01F0000EB3ECB5
:1022400001F0000EB3EC01F0000EB3EC01F0070E4C
:10225000B3EC01F0210EB3EC01F0AF0EB3EC01F0E2
:10226000640E33EC03F0800E026E400E096E216A9C
:1022700040C320F0066A056A200E016E100EF76E4C
:10228000F80EF66E0900F55003E0B3EC01F0FAD752
:102290000D0EB3EC01F00A0EB3EC01F0640E33EC5A
:1022A00003F0800E026E400E096E216A40C320F0DA
:1022B000066A056A200E016E110EF76E100EF66E9C
:1022C0000900F55003E0B3EC01F0FAD70D0EB3ECC2
:1022D00001F00A0EB3EC01F0640E33EC03F0800E53
:1022E000026E400E096E216A40C320F0066A056A3C
:1022F000200E016E110EF76E280EF66E0900F550D5
:1023000003E0B3EC01F0FAD70D0EB3EC01F00A0EC6
:10231000B3EC01F0640E33EC03F0800E026E400E5D
:10232000096E216A40C320F0066A056A200E016E1C
:10233000110EF76E400EF66E0900F55003E0B3EC97
:1023400001F0FAD70D0EB3EC01F00A0EB3EC01F078
:10235000640E33EC03F0800E026E400E096E216AAB
:1023600040C320F0066A056A200E016E110EF76E5A
:10237000580EF66E0900F55003E0B3EC01F0FAD701
:102380000D0EB3EC01F00A0EB3EC01F0640E33EC69
:1023900003F0800E026E400E096E216A40C320F0E9
:1023A000066A056A200E016E110EF76E700EF66E4B
:1023B0000900F55003E0B3EC01F0FAD70D0EB3ECD1
:1023C00001F00A0EB3EC01F02FEC49F003012A51A1
:1023D0000001E8A402D02FEC49F003012A510001CA
:1023E000E8A402D02FEC49F003013C510001E8B40D
:1023F0003CD003013D3500011CE2800E026E400E10
:10240000096E216A40C320F0066A056A200E016E3B
:10241000110EF76E880EF66E0900F55003E0B3EC6E
:1024200001F0FAD70D0EB3EC01F00A0EB3EC01F097
:102430001BD0800E026E400E096E216A40C320F050
:10244000066A056A200E016E110EF76EBA0EF66E60
:102450000900F55003E0B3EC01F0FAD70D0EB3EC30
:1024600001F00A0EB3EC01F03BD003013D35000151
:102470001CE2800E026E400E096E216A40C320F0FD
:10248000066A056A200E016E110EF76ED20EF66E08
:102490000900F55003E0B3EC01F0FAD70D0EB3ECF0
:1024A00001F00A0EB3EC01F01BD0800E026E400E5C
:1024B000096E216A40C320F0066A056A200E016E8B
:1024C000120EF76E040EF66E0900F55003E0B3EC41
:1024D00001F0FAD70D0EB3EC01F00A0EB3EC01F0E7
:1024E00003013C310001D8B0FEEC19F003012D6B63
:1024F000140E2C6F640E2E6F0001B4D1040E030174
:102500003A5D000106E2EA0E156E600E34EC03F04F
:10251000A9D103013D310001D8A05BD003013D35B5
:1025200000011CE2800E026E400E096E216A40C35B
:1025300020F0066A056A200E016E120EF76E1C0E60
:10254000F66E0900F55003E0B3EC01F0FAD70D0E7A
:10255000B3EC01F00A0EB3EC01F03BD0800E026E3A
:10256000400E096E216A40C320F0066A056A200EFB
:10257000016EB50EB3EC01F0620EB3EC01F0060E85
:10258000B3EC01F0570EB3EC01F0080EB3EC01F020
:10259000000EB3EC01F0010EB3EC01F0000EB3EC51
:1025A00001F0000EB3EC01F0000EB3EC01F0500EA0
:1025B000B3EC01F04F0EB3EC01F0540EB3EC01F0AC
:1025C000530EB3EC01F0AC0EB3EC01F0850EB3EC9E
:1025D00001F003013E31000120E32CEC37F004C38D
:1025E00034F003C333F002C332F001C331F0386A70
:1025F000376A366A7E0E356EE4EC05F0010807E0B6
:102600003A0E04011F6F980E1E6F000105D01D0EBB
:1026100004011F6F4C0E1E6F0001A20ED36ED288F4
:10262000C2901D0E03012D5D00010FE305E14D0E6B
:1026300003012C5D000109E31FC415F004011E51C4
:1026400034EC03F0000121EC1FF0130E03012D5DAB
:1026500000010FE305E1890E03012C5D000109E390
:102660001FC415F004011E5134EC03F0000121ECED
:102670001FF0090E03012D5D000116E305E1C50EF3
:1026800003012C5D000110E31FC415F004011E516D
:1026900034EC03F0000121EC1FF0640E0301295D0E
:1026A000000102E20301292B050E03012D5D00014B
:1026B00013E305E1DD0E03012C5D00010DE31FC4F2
:1026C00015F004011E5134EC03F0000121EC1FF061
:1026D00003012A9700010BD0040E0301295D0001BC
:1026E00004E303012A87000102D003012A970301B2
:1026F0002D53000107E1650E03012C5D000102E28C
:10270000000E01D0010E3A6E010E03012D5D000195
:1027100008E305E12C0E03012C5D000102E3000E2D
:1027200001D0010E3A16010E03012AB7000E3A1627
:10273000000112E01FC415F004011E5134EC03F037
:10274000000121EC1FF01FC415F004011E5134ECF0
:1027500003F0000121EC1FF0710E04011E5D146EE8
:10276000020E1F59156E35EC03F0D298D20ED36EBF
:10277000C28003013D310001D8A05BD003013D358B
:1027800000011CE2800E026E400E096E216A40C3F9
:1027900020F0066A056A200E016E120EF76E2A0EF0
:1027A000F66E0900F55003E0B3EC01F0FAD70D0E18
:1027B000B3EC01F00A0EB3EC01F03BD0800E026ED8
:1027C000400E096E216A40C320F0066A056A200E99
:1027D000016EB50EB3EC01F0620EB3EC01F0060E23
:1027E000B3EC01F0570EB3EC01F0080EB3EC01F0BE
:1027F000000EB3EC01F0010EB3EC01F0000EB3ECEF
:1028000001F0000EB3EC01F0000EB3EC01F0200E6D
:10281000B3EC01F04E0EB3EC01F0550EB3EC01F049
:10282000520EB3EC01F07B0EB3EC01F0C30EB3EC2F
:1028300001F0130E156E880E34EC03F0C8EC3FF077
:10284000000E03013CB1010E3A6E000E2AB7010ED4
:102850003A12000107E0FEEC19F0010E156EF40EBD
:1028600034EC03F042D8040E03013A5D00013CE36E
:10287000070E156ED00E34EC03F037D8FBEC36F0B3
:10288000130E03012D5D000106E307E1890E03012C
:102890002C5D000102E2000E01D0010E3A6E00C371
:1028A00034F0FFC233F0FEC232F0FDC231F09A0EB6
:1028B000386E990E376E190E366E7F0E356E1CEC23
:1028C00006F03A16000110E0070E156ED00E34EC3B
:1028D00003F0EBC21AF336C3EBF214EC1DF005D88B
:1028E0001AC3EBF214EC1DF009D603013E510001AE
:1028F000E8A80AD000EE45F0120EF76E360EF66E1E
:10290000B3EC04F0EE6AFAD003013D35000137E282
:10291000800E026E800E096E216A40C320F00B0EFD
:10292000066EB80E056E72EC01F0D8A042EF1CF0F6
:102930002408F9E172EC01F0D8A042EF1CF047083E
:10294000F2E172EC01F0D8A042EF1CF05008EBE18C
:1029500072EC01F0D8A042EF1CF04708E4E172EC01
:1029600001F0D8A042EF1CF04708DDE172EC01F065
:10297000D8A042EF1CF003011C6F000135D0800E7F
:10298000026E800E096E216A40C320F00B0E066EA7
:10299000B80E056E72EC01F0D8A042EF1CF02408CE
:1029A000F9E172EC01F0D8A042EF1CF04708F2E127
:1029B00072EC01F0D8A042EF1CF04E08EBE172EC93
:1029C00001F0D8A042EF1CF04708E4E172EC01F0FE
:1029D000D8A042EF1CF04708DDE172EC01F0D8A06E
:1029E00042EF1CF003011C6F010E0301256F1CC395
:1029F000F1F00001800E026E800E096E216A40C364
:102A000020F0066AC80E056E72EC01F0D8A06DD7F2
:102A100003011C6F00EEF1F025511CC3EBFF252BC9
:102A20002A0E1C5DD8A4010E3A6E4F0E255D010ED4
:102A3000D8B0000E3A160001DCE1800E026E800E66
:102A4000096E216A40C320F0050E396E020E086E31
:102A500008EC00F00301266FF36A00EEF1F0255157
:102A6000F3CFEBFF3D35000114E200EE45F0470ED9
:102A7000EE6E500EEE6E470EEE6EEE6E10EEF1F054
:102A8000550EE75204E0E6CFEEFFE82EFAD7EF6AE4
:102A900013D000EE45F0470EEE6E4E0EEE6E470E72
:102AA000EE6EEE6E10EEF1F0550EE75204E0E6CF5A
:102AB000EEFFE82EFAD7EF6A0201C06B03011B6B31
:102AC000000100EE45F00201C051EB500C6E2A0EE1
:102AD0000C5C00010CE000EE45F00201C051EB502F
:102AE0000C6E03011B1B0201C02B0001E9D703017F
:102AF0001B51265D0001D8A466EF1CF003013E5176
:102B00000001E8A80AD000EE9BF0120EF76E840ECA
:102B1000F66EB3EC04F0EE6A01D103013C51000102
:102B2000E8A430D103013D35000137E2800E026E8A
:102B3000800E096E216A40C320F00B0E066EB80E9F
:102B4000056E72EC01F0D8A042EF1CF02408F9E108
:102B500072EC01F0D8A042EF1CF04708F2E172ECF1
:102B600001F0D8A042EF1CF05008EBE172EC01F04C
:102B7000D8A042EF1CF05608E4E172EC01F0D8A0B6
:102B800042EF1CF05408DDE172EC01F0D8A042EFF6
:102B90001CF003011C6F000135D0800E026E800E08
:102BA000096E216A40C320F00B0E066EB80E056E4A
:102BB00072EC01F0D8A042EF1CF02408F9E172ECAD
:102BC00001F0D8A042EF1CF04708F2E172EC01F0EE
:102BD000D8A042EF1CF04E08EBE172EC01F0D8A057
:102BE00042EF1CF05608E4E172EC01F0D8A042EF8D
:102BF0001CF05408DDE172EC01F0D8A042EF1CF0AB
:102C000003011C6F010E0301256F1CC3F1F00001CD
:102C1000800E026E800E096E216A40C320F0066AA3
:102C2000C80E056E72EC01F0D8A068D703011C6FC6
:102C300000EEF1F025511CC3EBFF252B2A0E1C5D85
:102C4000D8A4010E3A6E4F0E255D010ED8B0000ECD
:102C50003A160001DCE1800E026E800E096E216AD8
:102C600040C320F0050E396E020E086E08EC00F02D
:102C70000301266FF36A00EEF1F02551F3CFEBFF6D
:102C80003D35000115E200EE9BF0470EEE6E500E52
:102C9000EE6E560EEE6E540EEE6E10EEF1F0550E18
:102CA000E75204E0E6CFEEFFE82EFAD7EF6A14D041
:102CB00000EE9BF0470EEE6E4E0EEE6E560EEE6E72
:102CC000540EEE6E10EEF1F0550EE75204E0E6CF32
:102CD000EEFFE82EFAD7EF6A0201C06B03011B6B0F
:102CE000000100EE9BF00201C051EB500C6E2A0E69
:102CF0000C5C00010CE000EE9BF00201C051EB50B7
:102D00000C6E03011B1B0201C02B0001E9D703015C
:102D10001B51265D0001D8A49AEF1CF000EEF1F0E3
:102D200010EE9BF0550EE75204E0E6CFEEFFE82EE2
:102D3000FAD7EF6A02EE1EF0EF6A02EE2EF0EF6AAB
:102D40000201CD6B0001DAEC1EF002EE1EF012EE75
:102D500044F0320EE75204E0E6CFEEFFE82EFAD759
:102D6000EF6A0201CD6B0001E0EC1EF002EE2EF0E6
:102D700012EE44F0320EE75204E0E6CFEEFFE82E0A
:102D8000FAD7EF6A0301386B00EEF1F010EE45F070
:102D9000550EE75204E0E6CFEEFFE82EFAD7EF6AD1
:102DA0000201CD6B0001DBEC1EF002014451BB6F50
:102DB000300EBB5D0001D8A45ED03A0E03012E5D3B
:102DC000000106E203012E2B000175EF14F052D032
:102DD00003012D530001D8A44DD0640E03012C5DD6
:102DE0000001D8B047D002EE3EF0300EEE6EEF6A32
:102DF0000201CD6B000106EC1FF000EEF1F00201C4
:102E0000CD51EBCF0CF00CC0DEF1CD2900EEF1F08E
:102E1000EBCF0CF00CC0DFF13A0E0101E06F020EB7
:102E20000201CD2500EEF1F0EBCF0CF00CC0E1F18A
:102E3000030ECD2500EEF1F0EBCF0CF00CC0E2F16B
:102E40003A0E0101E36F040E0201CD2500EEF1F010
:102E5000EBCF0CF00CC0E4F1050ECD2500EEF1F047
:102E6000EBCF0CF00CC0E5F10101E66B000116D9C7
:102E700075EF14F013D101EEDEF0EF6A01EEEEF023
:102E8000EF6A01EEFEF0EF6A02EE3EF0EF6A020139
:102E9000CD6B000106EC1FF000EEF1F00201CD5108
:102EA000EBCF0CF00CC0DEF1CD2900EEF1F0EBCF52
:102EB0000CF00CC0DFF13A0E0101E06F020E0201CE
:102EC000CD2500EEF1F0EBCF0CF00CC0E1F1030EDC
:102ED000CD2500EEF1F0EBCF0CF00CC0E2F13A0E94
:102EE0000101E36F040E0201CD2500EEF1F0EBCFFE
:102EF0000CF00CC0E4F1050ECD2500EEF1F0EBCFA7
:102F00000CF00CC0E5F10101E66B0201CD6B000194
:102F1000DFEC1EF001EEEEF012EE44F0080EE6CF0C
:102F2000EEFFE82EFCD7EF6A0201CD6B0001DEEC6C
:102F30001EF002EE44F0EECFF3FFEFCFF4FFF350BC
:102F4000530AF4101AE102EE44F02D0EEE6E11EE6B
:102F5000EEF00F0EE75204E0E6CFEEFFE82EFAD7D0
:102F6000EF6A01EEEEF012EE44F0320EE75204E0AA
:102F7000E6CFEEFFE82EFAD7EF6A0201CD6B000133
:102F8000DDEC1EF001EEFEF012EE44F0090EE6CF8D
:102F9000EEFFE82EFCD7EF6A0201CD6B0001DCECFE
:102FA0001EF002EE44F0EECFF3FFEFCFF4FFF3504C
:102FB000570AF4101AE102EE44F02D0EEE6E11EEF7
:102FC000FEF00F0EE75204E0E6CFEEFFE82EFAD750
:102FD000EF6A01EEFEF012EE44F0320EE75204E02A
:102FE000E6CFEEFFE82EFAD7EF6A0201CD6B0001C3
:102FF000DAEC1EF002EE3EF012EE44F0320EE75232
:1030000004E0E6CFEEFFE82EFAD7EF6A02EE3EF0DC
:1030100004EC00F003013A6F0201CD6B0001D8EC23
:103020001EF0040E03013A5D000114E302EE0EF0FF
:1030300012EE44F0320EE75204E0E6CFEEFFE82E47
:10304000FAD7EF6A02EE0EF004EC00F003012C6FE9
:1030500019C02DF30201FB2B000EFC23FCC211F062
:10306000FBC210F0030E156EE80E146E01EC04F0B6
:1030700019C0FCF218C0FBF203013C510001E8BC8E
:103080000DD002EE3EF0020E016E030E086EFCC281
:1030900019F0FBC218F0A7EC00F0EF6A03012E6BE9
:1030A000000E3CB7010E3A6E000E3CB3010E3A1210
:1030B0000001D8A4FBEC36F0000E03013DB3010E75
:1030C0003A6E000E3CB9010E3A12000104E05EECCB
:1030D0001DF0E4EC35F0C8EC3FF001EE47F0240EB3
:1030E000EE6EEE6EEE6EEE6E12EE77F0110EE752B1
:1030F00004E0E6CFEEFFE82EFAD72C0EEE6E12EECD
:103100003EF0050EE75204E0E6CFEEFFE82EFAD7D8
:103110002C0EEE6E11EEDEF00F0EE75204E0E6CF5D
:10312000EEFFE82EFAD72C0EEE6E11EEEEF00F0E3B
:10313000E75204E0E6CFEEFFE82EFAD72C0EEE6E53
:1031400011EEFEF00F0EE75204E0E6CFEEFFE82EA0
:10315000FAD72C0EEE6E12EE0EF00F0EE75204E0D0
:10316000E6CFEEFFE82EFAD7EF6A03012A510001FD
:10317000E8B6F5D003013E510001E8A617D025ECD2
:1031800044F001EE47F0EE50FEE1ED522C0EEE6EF3
:10319000020E016ED9C326F0D8C325F0D7C324F0A0
:1031A000D6C323F0010EE1EC00F0EF6A03013C51BD
:1031B0000001E8A41CD001EE47F0EE50FEE1ED5214
:1031C0002C0EEE6E12EE1EF00F0EE75204E0E6CF6C
:1031D000EEFFE82EFAD72C0EEE6E12EE2EF00F0E4A
:1031E000E75204E0E6CFEEFFE82EFAD7EF6A0301DC
:1031F0003C510001E8AA17D069EC36F001EE47F027
:10320000EE50FEE1ED522C0EEE6E020E016E0AC380
:1032100026F009C325F008C324F007C323F0010EEC
:10322000E1EC00F0EF6A03013D510001E8A215D086
:1032300001EE47F0EE50FEE1ED522C0EEE6E020E66
:10324000016E0EC326F00DC325F00CC324F00BC392
:1032500023F0010EE1EC00F0EF6A03013C350001C0
:1032600017E3B2EC36F001EE47F0EE50FEE1ED521E
:103270002C0EEE6E020E016E12C326F011C325F065
:1032800010C324F00FC323F0030EE1EC00F0EF6A4B
:1032900003013C510001E8A814D001EE47F0EE50C4
:1032A000FEE1ED522C0EEE6E020E016E16C326F0FC
:1032B00015C325F014C324F013C323F0E1EC00F090
:1032C000EF6A03013C510001E8A614D001EE47F07B
:1032D000EE50FEE1ED522C0EEE6E020E016E00C3BA
:1032E00026F0FFC225F0FEC224F0FDC223F0E1EC7F
:1032F00000F0EF6A03013E31000131E35DEC37F08D
:1033000003013E510001E8A214D001EE47F0EE5057
:10331000FEE1ED522C0EEE6E020E016E04C326F09D
:1033200003C325F002C324F001C323F0E1EC00F055
:10333000EF6A03013E510001E8A411D001EE47F00D
:10334000EE50FEE1ED522C0EEE6E020E016E086A9A
:1033500006C319F005C318F0A2EC00F0EF6A0301F0
:103360003D510001E8A413D056EC3CF001EE47F0CB
:10337000EE50FEE1ED522C0EEE6E12EE44F0320EE7
:10338000E75204E0E6CFEEFFE82EFAD7EF6A03013A
:103390001B6B01EE47F0E86AEE5202E0E83EFCD714
:1033A0000B6E040E0201CD6F0201CD510B5C0001CA
:1033B0000FE301EE47F00201CD51E926000EEA22AB
:1033C000EF500C6E03011B1B0201CD2B0001ECE33F
:1033D00001EE47F0EE50FEE1ED522A0EEE6E020EC7
:1033E000016E086E03011B5188EC00F00D0EEE6EAD
:1033F0000A0EEE6EEF6A000178EF1EF003012E6BED
:103400002A93300E0201BB6F03013D510001E8A871
:10341000CBD003013E510001E8A80AD000EEF1F044
:10342000120EF76E360EF66EB3EC04F0EE6AA7D00D
:10343000800E026E800E096E216A40C320F00B0ED2
:10344000066EB80E056E72EC01F0D8A0ADD024085F
:10345000FAE172EC01F0D8A0A7D04708F4E172ECD1
:1034600001F0D8A0A1D05008EEE172EC01F0D8A094
:103470009BD04708E8E172EC01F0D8A095D047084E
:10348000E2E172EC01F0D8A08FD003011C6F010EB5
:10349000256F1CC3F1F00001800E026E800E096ED4
:1034A000216A40C320F0066AC80E056E72EC01F076
:1034B000D8A075EF14F003011C6F00EEF1F0255158
:1034C0001CC3EBFF252B2A0E1C5DD8A4010E3A6EFF
:1034D0004F0E255D010ED8B0000E3A160001DBE15B
:1034E000800E026E800E096E216A40C320F0050E28
:1034F000396E020E086E08EC00F00301266FF36AC5
:1035000000EEF1F02551F3CFEBFF00EE45F0470E52
:10351000EE6E500EEE6E470EEE6EEE6E10EEF1F0A9
:10352000550EE75204E0E6CFEEFFE82EFAD7EF6A39
:103530000201C06B03011B6B000100EE45F00201AC
:10354000C051EB500C6E2A0E0C5C00010CE000EE3A
:1035500045F00201C051EB500C6E03011B1B020130
:10356000C02B0001E9D703011B51265D000107E0D4
:1035700003012E2B050E2E5D0001D8A04AD70201B3
:10358000CD6B0001DBEC1EF002014451BB6F300E2D
:10359000BB5D000109E103012A510001E8B204D03A
:1035A00003012A83000135D7C8EC3FF0939A8A9A29
:1035B00014DA31EC1DF00201C06B0001AA6A100E92
:1035C0000201C025A96ED8B0AA2AB0EC02F0EC6FB7
:1035D000C02B200EEC5D00010BE103012851050D0D
:1035E000F3CF14F0F4CF15F035EC03F00001E5D77C
:1035F0000201EC29010ED8A4000E3A6E100EC05D37
:10360000000102E2000E01D0010E3A1202E1DDD803
:10361000D4D703012A510001E8B682D003013D51FD
:103620000001E8AC30D0030E156EE80E34EC03F068
:1036300002EE44F0550EEE6E020E016E00C326F04F
:10364000FFC225F0FEC224F0FDC223F0E1EC00F041
:10365000560EEE6EEF6A0201C06B000102EE44F0FE
:103660000201C051EB500C6E0C5200010CE002EE56
:1036700044F00201C051EB50EC6F0001A6D80201EA
:10368000C02B0001EAD703013C510001E8A248D059
:1036900002EE2EF0020E016E0AC326F009C325F0D9
:1036A00008C324F007C323F0010EE1EC00F0EF6A39
:1036B00002012E510C6E2D0E0C5C000103E14E0E2A
:1036C00002012E6F0001030E156EE80E34EC03F0BC
:1036D00002EE44F0540EEE6E12EE2EF00F0EE75294
:1036E00004E0E6CFEEFFE82EFAD7430EEE6EEF6A67
:1036F0000201C06B000102EE44F00201C051EB5028
:103700000C6E0C5200010CE002EE44F00201C051BC
:10371000EB50EC6F000159D80201C02B0001EAD731
:10372000000E03013DB9010E3A6E000E2AB7010EDC
:103730003A120001D8B443D0300E0201BB5D000143
:103740003EE00201CD6B0001D8EC1EF002EE44F029
:1037500004EC00F003012C6F19C02DF3000156ECAE
:103760003CF002EE44F0EE50FEE1ED52200EEE6E23
:10377000020E016E086A2DC319F02CC318F0A7ECD5
:1037800000F0EF6A030E156EE80E34EC03F0020150
:10379000C06B000102EE44F00201C051EB500C6E10
:1037A0000C5200010CE002EE44F00201C051EB505B
:1037B000EC6F00010AD80201C02B0001EAD75BD9E7
:1037C000030E156EE80E34EF03F0410E0201EC5DBE
:1037D000000112E2246A8E0E0201EC25236ED8B09D
:1037E000242A2E0E235CEE6FAA6AEEC2A9FFB0EC6B
:1037F00002F0EB6F000110D0246A9E0E0201EC254E
:10380000236ED8B0242A410E235CEE6FAA6AEEC262
:10381000A9FFB0EC02F0EB6F0201EB510001E8BE32
:1038200026D0020E0201EB5D000121E3939A8A8A01
:103830000201EB3100010BE303012851030DF3CF2B
:1038400014F0F4CF15F035EC03F0000104D00301BF
:10385000285133EC03F00001939A8A9A030128510E
:1038600033EC03F0D8900201EB330001D5D703010C
:103870002851020DF3CF14F0F4CF15F035EC03F01E
:1038800000011200949494948B94640E33EC03F032
:1038900094840301382B060E385D000115E301EE18
:1038A00047F00D0EEE6E0A0EEE6E120EF76EAA0EB9
:1038B000F66EB3EC04F00D0EEE6E0A0EEE6EEF6ACD
:1038C0000301386B000114D275EF14F00301382B9B
:1038D000060E385D00012CE301EE47F00D0EEE6E92
:1038E0000A0EEE6E120EF76ECA0EF66EB3EC04F010
:1038F000240EEE6E470EEE6E500EEE6E470EEE6E1E
:10390000EE6E10EEF1F0550EE75204E0E6CFEEFF5A
:10391000E82EFAD7200EEE6EEE6E0D0EEE6E0A0E4B
:10392000EE6EEF6A0301386B000102EC3CF0E0D16F
:1039300075EF14F00301382B060E385D00012DE3FE
:1039400001EE47F00D0EEE6E0A0EEE6E120EF76EE1
:10395000CA0EF66EB3EC04F0240EEE6E470EEE6E59
:10396000500EEE6E560EEE6E540EEE6E10EEF1F040
:10397000550EE75204E0E6CFEEFFE82EFAD7200E10
:10398000EE6EEE6E0D0EEE6E0A0EEE6EEF6A030137
:10399000386B000102EC3CF0ABD175EF14F0050E72
:1039A0000201896F110E8A6F200E8B6F010E8C6FD2
:1039B0008D6B8A0E8E6F000153EF41F0050E0201F0
:1039C000896F110E8A6F200E8B6F010E8C6F8D6BBD
:1039D000880E8E6F000153EF41F0050E0201896FD2
:1039E000110E8A6F200E8B6F010E8C6F8D6B890EFE
:1039F0008E6F000153EF41F0080E0201896F130E24
:103A00008A6F040E8B6F150E8C6F210E8D6F200E3A
:103A10008E6F080E8F6F0B0E906F916B140E33EC40
:103A200003F0000155EF41F0050E0201896F110E00
:103A30008A6F220E8B6F010E8C6F8D6FEBC28EF230
:103A4000000153EF41F0050E0201896F110E8A6FDC
:103A50008B6B010E8C6F8D6BECC28EF2000153EFFD
:103A600041F0020E0201896F340E8A6F070E8B6FD0
:103A7000000153EF41F0020E0201896F340E8A6F8C
:103A8000010E8B6F000153EF41F0020E0201896FAE
:103A9000340E8A6F050E8B6F000153EF41F0060E56
:103AA0000201896F310E8A6F010E8B6F300E8C6FA1
:103AB0008D6B8E6B8F6B000153EF41F0020E020194
:103AC000896F340E8A6F030E8B6F000153EF41F044
:103AD000020E0201896F340E8A6F080E8B6F00018F
:103AE00053EF41F0080E0201896F320E8A6F8B6B23
:103AF0008C6B8D6B8E6B8F6B906B916B000153EFAA
:103B000041F0020E0201896F340E8A6F060E8B6F30
:103B1000000153EF41F0020E0201896F340E8A6FEB
:103B2000020E8B6F000153EF41F0D9C232F0D8C2C0
:103B300031F035EC08F0C8C238F0C7C237F0C6C261
:103B400036F0C5C235F094EC07F0E2EC07F0020164
:103B5000EF6F32C0F0F20001EFC2E7F2F0C2E8F21C
:103B6000060E0201896F110E8A6F200E8B6F020EF6
:103B70008C6F0D0E8D6FE8C28EF2E7C28FF20001DE
:103B800053EF41F0C8C226F0C7C225F0C6C224F0E8
:103B9000C5C223F030C332F02FC331F03DEC08F042
:103BA00034C02AF033C029F032C028F031C027F0E9
:103BB000346A336A326A7F0E316E2AC038F029C007
:103BC00037F028C036F027C035F0A0EC06F034C03E
:103BD0002AF033C029F032C028F031C027F0275234
:103BE000D8B43D84D8A4270626C038F025C037F0C5
:103BF00024C036F023C035F02AC034F029C033F099
:103C000028C032F027C031F094EC07F0E2EC07F066
:103C10000201F56F32C0F6F2F6C2EAF2F5C2E9F23D
:103C2000070E896F110E8A6F200E8B6F030E8C6F3B
:103C30000A0E8D6F8E6BEAC28FF2E9C290F200011C
:103C400053EF41F0050E0201896F110E8A6F200EAD
:103C50008B6F010E8C6F1A0E8D6F8E6B000153EC03
:103C600041F0136A080E126E116A106A1B6A1A6A12
:103C7000196ACEC218F053EC04F013C0DFF212C080
:103C8000DEF211C0DDF210C0DCF2DFC213F0DEC2E2
:103C900012F0DDC211F0DCC210F01B681A6819685E
:103CA000186A76EC03F013C0DFF212C0DEF211C026
:103CB000DDF210C0DCF2DEC241F3DDC242F3DCC251
:103CC00043F3030E03014117060E0201896F110E23
:103CD0008A6F200E8B6F030E8C6F1B0E8D6F41C38E
:103CE0008EF242C38FF243C390F2000153EF41F0D2
:103CF000939A8A8A54DEB5DE640E33EC03F0020137
:103D0000C06B000101EE47F00201C051E926000E30
:103D1000EA22EF500C6E000E0C52D8A4010E3A6E3F
:103D2000960EC05D010ED8B0000E3A16000110E0EC
:103D300001EE47F00201C051E926000EEA22EF50E1
:103D40000301276F000108D80201C02B0001D9D759
:103D5000640E33EC03F08FD6939A8A9AF8C211F06E
:103D60000201F75141EC03F0010E03011C6F030146
:103D70001C51335D000112E3030127B1818A27A1A1
:103D8000819AF8C211F00201F75141EC03F0D8908A
:103D90000301273303011C2B0001E9E3939A8A8A6C
:103DA000FAC211F00201F95141EC03F000011200D6
:103DB0002DD82CD82BD82AD829D828D827D826D8F7
:103DC00025D80201C06B000100EEF1F00201CD51D7
:103DD000EB500C6E2C0E0C5C00010FE000EEF1F0CD
:103DE0000201CD51EBCF0CF002EE44F0C0510CC0FB
:103DF000EBFFC02BCD2B0001E6D7F36A02EE44F0B7
:103E00000201C051F3CFEBFF0001120000EEF1F010
:103E10000201CD51EB500C6E2C0E0C5CD8A4010E9F
:103E20003A6E500ECD5D010ED8B0000E3A1600016C
:103E300004E00201CD2B0001E9D70201CD2B0001E6
:103E40001200939A8A8AEDEC1CF00BDE1D0E116EA7
:103E50004C0E41EC03F0939A8A9A1D0E116E4C0E93
:103E600041EC03F0939A8A8A1D0E116E4C0E41ECC0
:103E700003F001D6D7C2E6F2D6C2E5F2D5C2E4F22B
:103E8000D4C2E3F2640E33EC03F0949A8B8A020EF0
:103E9000156E580E34EC03F0949A8B9A949E8B9E78
:103EA000810E026E010E096E810E036E040E046E09
:103EB000010E0A6E106E08EC03F0949E8B8EC80EF5
:103EC00033EC03F0070E0201896F020E8A6F010EB8
:103ED0008B6F8C6BE6C28DF2E5C28EF2E4C28FF27C
:103EE000E3C290F203013D510001E8A603D0010EA8
:103EF00002018C6F000155EC41F0140E33EC03F01D
:103F0000040E0201896F200E8A6F8B6B8C6B8D6B98
:103F1000000155EC41F0140E33EC03F0FCEC1CF006
:103F2000CEEC41F002DE2EDE080E0201CF250301A9
:103F30001C6F050E0201896F110E8A6F200E8B6FA8
:103F4000010E8C6F510E8D6F1CC38EF2000153EC6D
:103F500041F0050E0201896F110E8A6F220E8B6FE0
:103F6000010E8C6F8D6B080E8E6F000153EC41F0CB
:103F700014EC1DF003013D510001E8A602D002013E
:103F8000EC6B000123EC1DF0050E0201896F110E90
:103F90008A6F8B6B010E8C6F8D6F8E6F000153EFEC
:103FA00041F0AE6A0D0E28EC02F0120EF76EE00E34
:103FB000F66E20EC02F0016A086A196A040E186EA7
:103FC000A7EC00F02E0E28EC02F0010E086E2D0E6C
:103FD000A5EC00F0120EF76EF40EF66E20EC02F077
:103FE0000D0E28EC02F0130E096E880E026EFBEC2B
:103FF00001F0D8A0BDEF0FF003013B6F120EF76E7A
:10400000FE0EF66E20EC02F00D0E28EC02F0630EB0
:1040100028EC02F06D0E28EC02F0640E28EC02F0A1
:104020003E0E28EC02F0000103D86ED8D1D8FBD7A1
:10403000130E096E880E026EFBEC01F0F9E303012A
:104040003B6F3B5128EC02F00D0E3B5D010ED8A4F6
:10405000000E3A6E0A0E3B5D010ED8A4000E3A1215
:104060000001D8A41200010E0301256F3BC3F1F03B
:104070000001130E096E880E026EFBEC01F03AE3AC
:1040800003013B6F3B5128EC02F0080E3B5D000141
:1040900008E103012553000102E0030125070001A7
:1040A000E7D70D0E03013B5D010ED8A4000E3A6E5A
:1040B0000A0E3B5D010ED8A4000E3A122529010E0E
:1040C000D8A4000E3A1200010BE00D0EF36E00EEC4
:1040D000F1F003012551F3CFEBFF0001120006D0F0
:1040E00000EEF1F0030125513BC3EBFF0301252B4B
:1040F0000001BED70D0EF36E00EEF1F00301255165
:10410000F3CFEBFF000112000201CD6B000100EEC6
:10411000F1F00201CD51EB500C6E200E0C5CD8A4D6
:10412000010E3A6E00EEF1F0CD51EB500C6E0D0E1B
:104130000C5CD8A4010E3A16FD0ECD5D010ED8B070
:10414000000E3A1600013AE000EEF1F00201CD5106
:10415000EB500C6E610E0C5C000ED8B0010E3A6E86
:1041600000EEF1F0CD51EB500C6E7B0E0C5C0001BB
:1041700002E3000E01D0010E3A160EE000EEF1F05F
:104180000201CD51EB500E6EDF0E0E140C6E00EEE0
:10419000F1F0CD510CC0EBFF000100EEF1F0020197
:1041A000CD51EBCF0CF001EE47F0CD51E926000EDA
:1041B000EA220CC0EFFFCD2B0001A8D701EE47F09B
:1041C0000201CD51E926000EEA22EF6A0001120039
:1041D000F1510C6E0A0E0C5C010ED8A4000E3A6E62
:1041E000F1510C6E0D0E0C5C010ED8A4000E3A12AB
:1041F000D8A41200130EF76E120EF66E01EE47F001
:10420000BBEC04F002E144D228D2130EF76E180E74
:10421000F66E01EE47F0BBEC04F009E0130EF76E0A
:104220001C0EF66E01EE47F0BBEC04F003E108EF64
:104230002DF013D2130EF76E240EF66E01EE47F03A
:10424000BBEC04F009E0130EF76E280EF66E01EEDB
:1042500047F0BBEC04F003E165EF25F0FED1130E4F
:10426000F76E2E0EF66E01EE47F0BBEC04F003E1A4
:1042700035EF25F0F2D1130EF76E360EF66E01EE25
:1042800047F0BBEC04F003E14DEF25F0E6D1130E4F
:10429000F76E3C0EF66E01EE47F0BBEC04F003E166
:1042A0003AEF2DF0DAD1130EF76E420EF66E01EEF4
:1042B00047F0BBEC04F009E0130EF76E460EF66E05
:1042C00001EE47F0BBEC04F003E1E1EF29F0C5D1CA
:1042D000130EF76E500EF66E01EE47F0BBEC04F0D5
:1042E00009E0130EF76E540EF66E01EE47F0BBECCC
:1042F00004F003E118EF2CF0B0D1130EF76E5E0E50
:10430000F66E01EE47F0BBEC04F009E0130EF76E19
:10431000640EF66E01EE47F0BBEC04F003E14CEFE7
:104320002CF09BD1130EF76E6A0EF66E01EE47F07D
:10433000BBEC04F003E18AEF2CF08FD1130EF76E83
:10434000700EF66E01EE47F0BBEC04F003E19AEF5D
:104350002CF083D1130EF76E760EF66E01EE47F059
:10436000BBEC04F009E0130EF76E7C0EF66E01EE66
:1043700047F0BBEC04F003E163EF2DF06ED1130EB8
:10438000F76E820EF66E01EE47F0BBEC04F009E02A
:10439000130EF76E880EF66E01EE47F0BBEC04F0DC
:1043A00003E1D6EF2CF059D1130EF76E8E0EF66E98
:1043B00001EE47F0BBEC04F003E1D5EF24F04DD162
:1043C000130EF76E940EF66E01EE47F0BBEC04F0A0
:1043D00003E1EDEF24F041D1130EF76E9A0EF66E65
:1043E00001EE47F0BBEC04F003E175EF24F035D1AA
:1043F000130EF76EA00EF66E01EE47F0BBEC04F064
:1044000003E105EF25F029D1130EF76EA60EF66E27
:1044100001EE47F0BBEC04F003E11DEF25F01DD1E8
:10442000130EF76EAE0EF66E01EE47F0BBEC04F025
:1044300002E1D9D112D1130EF76EB60EF66E01EE6F
:1044400047F0BBEC04F009E0130EF76EBC0EF66EFD
:1044500001EE47F0BBEC04F002E17DD1FED0130E7B
:10446000F76EC60EF66E01EE47F0BBEC04F002E10B
:104470008AD1F3D0130EF76ECC0EF66E01EE47F034
:10448000BBEC04F002E197D1E8D0130EF76ED40E26
:10449000F66E01EE47F0BBEC04F002E1BCD1DDD0DA
:1044A000130EF76EDC0EF66E01EE47F0BBEC04F077
:1044B00002E133D2D2D0130EF76EE20EF66E01EEA9
:1044C00047F0BBEC04F002E1F8D1C7D0130EF76E51
:1044D000E80EF66E01EE47F0BBEC04F003E195EF59
:1044E00025F0BBD0130EF76EEE0EF66E01EE47F020
:1044F000BBEC04F003E13DEF26F0AFD0130EF76EF6
:10450000F40EF66E01EE47F0BBEC04F003E1C7EFEA
:104510002AF0A3D0130EF76EF80EF66E01EE47F0F8
:10452000BBEC04F003E17DEF25F097D0130EF76E9E
:10453000FE0EF66E01EE47F0BBEC04F003E190EFE7
:104540002BF08BD0140EF76E060EF66E01EE47F0D0
:10455000BBEC04F003E15CEF2FF07FD0140EF76E9C
:104560000C0EF66E01EE47F0BBEC04F003E12EEF0B
:104570002EF073D0140EF76E120EF66E01EE47F0A9
:10458000BBEC04F002E19ED068D0140EF76E180E5A
:10459000F66E01EE47F0BBEC04F003E1AFEF25F05F
:1045A0005CD0140EF76E1E0EF66E01EE47F0BBECFB
:1045B00004F003E1DDEF25F050D0140EF76E240E69
:1045C000F66E01EE47F0BBEC04F002E195D045D069
:1045D000140EF76E2C0EF66E01EE47F0BBEC04F0F5
:1045E00003E1ECEF2DF039D0140EF76E360EF66EB7
:1045F00001EE47F0BBEC04F003E164EF2EF02DD0A8
:10460000140EF76E3C0EF66E01EE47F0BBEC04F0B4
:1046100002E19BD122D0140EF76E420EF66E01EE2F
:1046200047F0BBEC04F002E1A8D117D0140EF76EEE
:10463000480EF66E01EE47F0BBEC04F003E1FFEF2D
:104640002DF00BD0140EF76E4C0EF66E01EE47F007
:10465000BBEC04F0D8B41CEF2EF0140EF76E520E23
:10466000F66E20EC02F00D0E28EC02F0630E28EC42
:1046700002F06D0E28EC02F0640E28EC02F03E0E03
:1046800028EC02F0640E33EC03F074CF1CF312003C
:10469000B9EC30F0EEEC2EF003012A310001D8B075
:1046A000FFEF30F003012A31E832D8B03C81D8A0C6
:1046B0003C91AA6A7E0EA96E3C51B7EC02F0000153
:1046C0001EEF31F0B9EC30F0EEEC2EF003012A31A0
:1046D0000001D8B0FFEF30F003012A31E832D8B042
:1046E0003D81D8A03D91AA6A7F0EA96E3D51B7ECDD
:1046F00002F000011EEF31F035EC31F003011D51E5
:10470000300A1E11000105E1BC0E0301406F0001DB
:1047100018D003011D51600A1E11000105E1500E61
:104720000301406F00010DD003011D51C00A1E118D
:10473000000105E11E0E0301406F000102D0FFEFF2
:1047400030F0AA6A870EA96E03014051B7EC02F05F
:1047500000011EEF31F0EEEC2EF003012A310001D2
:10476000D8B0FFEF30F003012A31E832D8B03E87ED
:10477000D8A03E97AA6A800EA96E3E51B7EC02F00F
:1047800000011EEF31F0EEEC2EF003012A310001A2
:10479000D8B0FFEF30F003012A31E832D8B03D8DB8
:1047A000D8A03D9DAA6A7F0EA96E3D51B7EC02F0DC
:1047B00000011EEF31F0EEEC2EF003012A31000172
:1047C000D8B0FFEF30F003012A31E832D8B03C8393
:1047D000D8A03C93AA6A7E0EA96E3C51B7EC02F0B9
:1047E00000011EEF31F0EEEC2EF003012A31000142
:1047F000D8B0FFEF30F003012A31E832D8B03C8F57
:10480000D8A03C9FAA6A7E0EA96E3C51B7EC02F07C
:1048100000011EEF31F0EEEC2EF003012A31000111
:10482000D8B0FFEF30F003012A31E832D8B03C8530
:10483000D8A03C95AA6A7E0EA96E3C51B7EC02F056
:104840003C510001E8B41CD0800E026E400E096E8F
:10485000216A40C320F0066A056A200E016E110E1F
:10486000F76E880EF66E0900F55003E0B3EC01F028
:10487000FAD70D0EB3EC01F00A0EB3EC01F01BD029
:10488000800E026E400E096E216A40C320F0066A57
:10489000056A200E016E110EF76ED20EF66E09003B
:1048A000F55003E0B3EC01F0FAD70D0EB3EC01F0D4
:1048B0000A0EB3EC01F01EEF31F0EEEC2EF0030126
:1048C0002A310001D8B0FFEF30F003012A31E8327D
:1048D000D8B03C89D8A03C99AA6A7E0EA96E3C51FA
:1048E000B7EC02F000011EEF31F0EEEC2EF0030108
:1048F0002A310001D8B0FFEF30F003012A31E8324D
:10490000D8B03E85D8A03E95AA6A7E0EA96E3C51CD
:10491000B7EC02F000011EEF31F0EEEC2EF00301D7
:104920002A310001D8B0FFEF30F003012A31E8321C
:10493000D8B03C87D8A03C97AA6A7E0EA96E3C519D
:10494000B7EC02F000011EEF31F0EEEC2EF00301A7
:104950002A310001D8B0FFEF30F003012A31E832EC
:10496000D8B03E89D8A03E99AA6A800EA96E3E5161
:10497000B7EC02F000011EEF31F0EEEC2EF0030177
:104980002A310001D8B0FFEF30F003012A31E832BC
:10499000D8B03D8FD8A03D9FAA6A7F0EA96E3D5129
:1049A000B7EC02F000011EEF31F0EEEC2EF0030147
:1049B0002A310001D8B0FFEF30F003012A31E8328C
:1049C000D8B03E81D8A03E91AA6A800EA96E3E5111
:1049D000B7EC02F000011EEF31F0EEEC2EF0030117
:1049E0002A310001D8B0FFEF30F003012A31E8325C
:1049F000D8B03E83D8A03E93AA6A7F0EA96E3D51DF
:104A0000B7EC02F000011EEF31F0EEEC2EF00301E6
:104A10002A310001D8B0FFEF30F003012A31E8322B
:104A2000D8B03C8BD8A03C9BAA6A7E0EA96E3C51A4
:104A3000B7EC02F000011EEF31F0EEEC2EF00301B6
:104A40002A310001D8B0FFEF30F003012A31E832FB
:104A5000D8B03D83D8A03D93AA6A7F0EA96E3D5180
:104A6000B7EC02F000011EEF31F0EEEC2EF0030186
:104A70002A310001D8B0FFEF30F003012A31E832CB
:104A8000D8B03D85D8A03D95AA6A7F0EA96E3D514C
:104A9000B7EC02F000011EEF31F0EEEC2EF0030156
:104AA0002A310001D8B0FFEF30F003012A31E8329B
:104AB000D8B03D8BD8A03D9BAA6A7F0EA96E3D5110
:104AC000B7EC02F000011EEF31F0EEEC2EF0030126
:104AD0002A310001D8B0FFEF30F003012A31E8326B
:104AE000D8B03D89D8A03D99AA6A7F0EA96E3D51E4
:104AF000B7EC02F000011EEF31F0EEEC2EF00301F6
:104B00002A310001D8B0FFEF30F003012A31E8323A
:104B1000D8B03D87D8A03D97AA6A7F0EA96E3D51B7
:104B2000B7EC02F000011EEF31F0EEEC2EF00301C5
:104B30002A310001D8B0FFEF30F0E86A03012AB350
:104B4000010E010AD8B43C9DD8A43C8DAA6A7E0E01
:104B5000A96E3C51B7EC02F000011EEF31F0B9EC48
:104B600030F0F1510C6E300E0C5CD8B4AEEF37F073
:104B7000F1510C6E310E0C5CD8B45EEF38F0F1518F
:104B80000C6E320E0C5CD8B45FEF39F0F1510C6E44
:104B9000330E0C5CD8B449EF3AF0F1510C6E340E80
:104BA0000C5CD8B4EEEF3AF0F1510C6E350E0C5CA3
:104BB000D8B447EF3BF0FFEF30F0140EF76E680EFD
:104BC000F66E20EC02F00D0E28EC02F0939A8A8A21
:104BD000DEEC1CF04FEC1DF00B0E096EB80E026EF1
:104BE000FBEC01F0F9E303011C6F550E1C5D010E97
:104BF000D8A4000E3A6E750E1C5D010ED8A4000EEE
:104C00003A12000106E00201EC53000102E0020149
:104C1000EC07440E03011C5D010ED8A4000E3A6E91
:104C2000640E1C5D010ED8A4000E3A12000107E0CC
:104C30007F0E0201EC5D000102E20201EC2B450E49
:104C400003011C5D010ED8A4000E3A6E650E1C5DBA
:104C5000010ED8A4000E3A1200010CE03BEC1DF04E
:104C6000AA6A880EA96E0201EC51B7EC02F00001AD
:104C70001EEF31F023EC1DF0AFD70D0E28EC02F043
:104C8000140EF76E8C0EF66E20EC02F003013D352B
:104C9000000107E34F0E28EC02F04E0E28EC02F064
:104CA00008D04F0E28EC02F0460E28EC02F028EC5B
:104CB00002F00D0E28EC02F0140EF76E940EF66E54
:104CC00020EC02F003013E31000107E34F0E28EC17
:104CD00002F04E0E28EC02F008D04F0E28EC02F045
:104CE000460E28EC02F028EC02F00D0E28EC02F043
:104CF000140EF76EA00EF66E20EC02F003013C518C
:104D00000001E8AA07D04F0E28EC02F04E0E28EC66
:104D100002F008D04F0E28EC02F0460E28EC02F00C
:104D200028EC02F00D0E28EC02F0140EF76EAE0E19
:104D3000F66E20EC02F003013D510001E8A207D01D
:104D40004F0E28EC02F04E0E28EC02F008D04F0E69
:104D500028EC02F0460E28EC02F028EC02F00D0ED2
:104D600028EC02F0140EF76EC40EF66E20EC02F082
:104D700003013C35000107E34F0E28EC02F04E0E14
:104D800028EC02F008D04F0E28EC02F0460E28EC7A
:104D900002F028EC02F00D0E28EC02F0140EF76E73
:104DA000DA0EF66E20EC02F003013C510001E8A49B
:104DB00007D04F0E28EC02F04E0E28EC02F008D07F
:104DC0004F0E28EC02F0460E28EC02F028EC02F020
:104DD0000D0E28EC02F0140EF76EEA0EF66E20ECC3
:104DE00002F003013C510001E8A607D04F0E28EC69
:104DF00002F04E0E28EC02F008D04F0E28EC02F024
:104E0000460E28EC02F028EC02F00D0E28EC02F021
:104E1000140EF76EF60EF66E20EC02F003013C5114
:104E20000001E8A807D04F0E28EC02F04E0E28EC47
:104E300002F008D04F0E28EC02F0460E28EC02F0EB
:104E400028EC02F00D0E28EC02F0150EF76E060E9F
:104E5000F66E20EC02F003013E510001E8A207D0FB
:104E60004F0E28EC02F04E0E28EC02F008D04F0E48
:104E700028EC02F0460E28EC02F028EC02F00D0EB1
:104E800028EC02F0150EF76E140EF66E20EC02F010
:104E900003013E510001E8A407D04F0E28EC02F0B8
:104EA0004E0E28EC02F008D04F0E28EC02F0460E11
:104EB00028EC02F028EC02F00D0E28EC02F0150EA2
:104EC000F76E220EF66E20EC02F003013C51000159
:104ED000E8BC07D04F0E28EC02F04E0E28EC02F092
:104EE00008D04F0E28EC02F0460E28EC02F028EC19
:104EF00002F00D0E28EC02F0430E28EC02F0570EE3
:104F000028EC02F0490E28EC02F0440E28EC02F0E6
:104F1000200E28EC02F003013C31000109E24F0EA3
:104F200028EC02F0460E28EC02F028EC02F006D045
:104F30004F0E28EC02F04E0E28EC02F00D0E28EC7D
:104F400002F0150EF76E2C0EF66E20EC02F0030147
:104F50003D510001E8AC07D04F0E28EC02F04E0E98
:104F600028EC02F008D04F0E28EC02F0460E28EC98
:104F700002F028EC02F00D0E28EC02F0150EF76E90
:104F8000340EF66E20EC02F003013C510001E8A261
:104F900007D04F0E28EC02F04E0E28EC02F008D09D
:104FA0004F0E28EC02F0460E28EC02F028EC02F03E
:104FB0000D0E28EC02F0150EF76E3C0EF66E20EC8E
:104FC00002F003013D510001E8A407D04F0E28EC88
:104FD00002F04E0E28EC02F008D04F0E28EC02F042
:104FE000460E28EC02F028EC02F00D0E28EC02F040
:104FF000150EF76E460EF66E20EC02F003013D51E1
:105000000001E8AA07D04F0E28EC02F04E0E28EC63
:1050100002F008D04F0E28EC02F0460E28EC02F009
:1050200028EC02F00D0E28EC02F0150EF76E4E0E75
:10503000F66E20EC02F003013D510001E8A807D014
:105040004F0E28EC02F04E0E28EC02F008D04F0E66
:1050500028EC02F0460E28EC02F028EC02F00D0ECF
:1050600028EC02F0150EF76E560EF66E20EC02F0EC
:1050700003013E510001E8A607D04F0E28EC02F0D4
:105080004E0E28EC02F008D04F0E28EC02F0460E2F
:1050900028EC02F028EC02F00D0E28EC02F0150EC0
:1050A000F76E600EF66E20EC02F003013D31000158
:1050B00007E34F0E28EC02F04E0E28EC02F008D069
:1050C0004F0E28EC02F0460E28EC02F028EC02F01D
:1050D0000D0E28EC02F0150EF76E680EF66E20EC41
:1050E00002F003011E6B1D6B1EC320F31DC31FF3D3
:1050F000040E0301205D000115E220C3AAFF1FC3B7
:10510000A9FFB0EC02F003011C6F1C2900010AE0AA
:1051100003011C5128EC02F003011F2B000E202379
:105120000001E6E30D0E28EC02F0150EF76E700E8E
:10513000F66E20EC02F003011E6B100E1D6F1EC3F5
:1051400020F31DC31FF3040E0301205D000115E2CF
:1051500020C3AAFF1FC3A9FFB0EC02F003011C6F1C
:105160001C2900010AE003011C5128EC02F0030194
:105170001F2B000E20230001E6E30D0E28EC02F0A9
:10518000150EF76E7A0EF66E20EC02F0016A086AD0
:10519000D3C226F0D2C225F0D1C224F0D0C223F06F
:1051A00040EC01F0200E28EC02F0480E28EC02F052
:1051B0007A0E28EC02F00D0E28EC02F0150EF76EB8
:1051C000860EF66E20EC02F0016A086A30C319F010
:1051D0002FC318F0A7EC00F0200E28EC02F0480EC8
:1051E00028EC02F07A0E28EC02F00D0E28EC02F00A
:1051F000150EF76E920EF66E20EC02F0016A086A48
:1052000032C319F031C318F0A7EC00F0200E28ECDF
:1052100002F0420E28EC02F0640E28EC02F00D0EB3
:1052200028EC02F0150EF76E9A0EF66E20EC02F0E6
:10523000016A03013351A4EC00F00D0E28EC02F0DA
:10524000150EF76EA60EF66E20EC02F0016A3451D0
:10525000A4EC00F00D0E28EC02F0150EF76EB20E65
:10526000F66E20EC02F0016A3F51A4EC00F0200E33
:1052700028EC02F06D0E28EC02F0570E28EC02F03C
:105280000D0E28EC02F0150EF76EBE0EF66E20EC39
:1052900002F0016A3551A4EC00F0200E28EC02F077
:1052A000570E28EC02F0500E28EC02F04D0E28ECC0
:1052B00002F00D0E28EC02F0150EF76ECC0EF66E15
:1052C00020EC02F0016A086AD9C219F0D8C218F0BD
:1052D000A2EC00F0200E28EC02F0480E28EC02F0C0
:1052E0007A0E28EC02F00D0E28EC02F03D51000180
:1052F000E8A606D0540E28EC02F0430E28EC02F08B
:10530000150EF76EDC0EF66E20EC02F0016A086AEC
:10531000D7C226F0D6C225F0D5C224F0D4C223F0DD
:1053200040EC01F0200E28EC02F0480E28EC02F0D0
:105330007A0E28EC02F00D0E28EC02F0870EAEEC8F
:1053400002F00301406F150EF76EEC0EF66E20ECC6
:1053500002F0A10E405D000109E3150EF76EF40E98
:10536000F66E20EC02F00D0E28EC02F04B0E03015D
:10537000405D000102E2000E01D0010E3A6E640EA3
:105380000301405D010ED8B0000E3A16000109E09D
:10539000150EF76EFC0EF66E20EC02F00D0E28ECEA
:1053A00002F02A0E0301405D000109E2160EF76EBD
:1053B000040EF66E20EC02F00D0E28EC02F01EEF4B
:1053C00031F035EC31F0F4C2D3F2F3C2D2F2F2C2D2
:1053D000D1F2F1C2D0F2C00E0201D05DCB0ED15994
:1053E000170ED259070ED3590001D8B073D002015D
:1053F000C06B150E0201C05D00010EE200EEF1F07F
:105400000201C051EB500C6E0D0E0C5C000104E06B
:105410000201C02B0001EDE3090E0201C05D000195
:105420000BE2300EF36E00EEF1F00201C051F3CF4B
:10543000EBFFC02B0001F0D70D0EFA6F0201D36B0A
:10544000D26BD16BD06BC06B090E0201C05D000145
:10545000D8B040D0266A256A246A0A0E236E26C078
:1054600013F025C012F024C011F023C010F0D3C2F5
:105470001BF0D2C21AF0D1C219F0D0C218F053EC0E
:1054800004F013C026F012C025F011C024F010C0A3
:1054900023F000EEF1F00201C051EB500C6E2A6ACD
:1054A000296A286A0CC027F00F0E27142A6A296A75
:1054B000286A276E2324D06F28502420D16F2950CA
:1054C0002520D26F2A502620D36F0201C02B000165
:1054D000D8A0BAD7070E0201D35D000114E311E191
:1054E000170E0201D25D00010EE30BE1CB0E0201AB
:1054F000D15D000108E305E1C00E0201D05D0001AD
:1055000002E3000E01D0010E3A6E810E0201D05D61
:10551000D90ED1599F0ED259380ED359000102E24B
:10552000000E01D0010E3A12D8A4FFEF30F00201B4
:10553000C06B0F0E0201C05D00011AE200EEF1F037
:105540000201C051EB5003011C6F0D0E1C5D0001E8
:105550000FE0AA6A1E0E0201C025A96ED8B0AA2AC1
:1055600003011C51B7EC02F00201C02B0001E1E382
:10557000AA6A1E0E0201C025A96ED8B0AA2AFF0E83
:10558000B7EC02F00001CEEC41F01EEF31F035EC4B
:1055900031F0F4C2D7F2F3C2D6F2F2C2D5F2F1C2C0
:1055A000D4F2800E0201D45D960ED559980ED659CC
:1055B000000ED7590001D8B073D00201C06B150E90
:1055C0000201C05D00010EE200EEF1F00201C051E7
:1055D000EB500C6E0D0E0C5C000104E00201C02BC0
:1055E0000001EDE3080E0201C05D00010BE2300E88
:1055F000F36E00EEF1F00201C051F3CFEBFFC02BD0
:105600000001F0D70D0EFA6F0201D76BD66BD56B88
:10561000D46BC06B090E0201C05D0001D8B040D050
:10562000266A256A246A0A0E236E26C013F025C056
:1056300012F024C011F023C010F0D7C21BF0D6C264
:105640001AF0D5C219F0D4C218F053EC04F013C00C
:1056500026F012C025F011C024F010C023F000EE97
:10566000F1F00201C051EB500C6E2A6A296A286AD7
:105670000CC027F00F0E27142A6A296A286A276EA1
:105680002324D46F28502420D56F29502520D66F8D
:105690002A502620D76F0201C02B0001D8A0BAD70C
:1056A000000E0201D75D000114E311E1980E020122
:1056B000D65D00010EE30BE1960E0201D55D0001FF
:1056C00008E305E1800E0201D45D000102E3000E53
:1056D00001D0010E3A6EC10E0201D45D0E0ED559F5
:1056E000160ED659020ED759000102E2000E01D063
:1056F000010E3A12D8A4FFEF30F0AA6A810EA96E0B
:105700000201D451B7EC02F0D551B7EC02F0D651FA
:10571000B7EC02F0D751B7EC02F000011EEF31F008
:10572000B9EC30F00201D96BD86B03012A93000168
:10573000F1510C6E2D0E0C5C02E103012A83020173
:10574000C06B0201C05103012AB3010F00EEF1F05A
:10575000EB500C6E0D0E0C5C000130E00201C051EC
:1057600003012AB3010F00EEF1F0EB501C6F246A25
:105770000A0E236E24C011F02350106E0201D803CC
:10578000F3CF23F0F4CF24F01150D803F3502426A4
:105790001050D903F35024261CC327F0286A27BED3
:1057A00028680F0E2716000E281627502324D86FBE
:1057B00028502420D96FC02B0001C3D703012A51E0
:1057C0000001E8A204D00201D86DE86AD9570201AD
:1057D000D9AF06D0D00ED85D8A0ED959000102E3A8
:1057E000000E01D0010E3A6E0201D9BF0AD0750E2B
:1057F000D95D07E3000107E1310E0201D85D000128
:1058000002E2000E01D0010E3A120001D8A4FFEF0F
:1058100030F0AA6A850EA96E0201D851B7EC02F0E9
:10582000D951B7EC02F0000195EC1DF01EEF31F0FC
:1058300035EC31F0F2C230F3F1C22FF30201C06B4C
:105840000F0E0201C05D00011AE200EEF1F002014C
:10585000C051EB5003011C6F0D0E1C5D00010FE0E9
:10586000AA6A2E0E0201C025A96ED8B0AA2A030189
:105870001C51B7EC02F00201C02B0001E1E3AA6A5F
:105880002E0E0201C025A96ED8B0AA2AFF0EB7ECD1
:1058900002F000011EEF31F035EC31F0F2C232F3CC
:1058A000F1C231F30201C06B0F0E0201C05D0001B5
:1058B00024E200EEF1F00201C051EB5003011C6F35
:1058C0000D0E1C5D010ED8A4000E3A6E2E0E1C5D4E
:1058D000010ED8A4000E3A1200010FE1AA6A3E0E92
:1058E0000201C025A96ED8B0AA2A03011C51B7EC49
:1058F00002F00201C02B0001D7E3AA6A3E0E0201AA
:10590000C025A96ED8B0AA2AFF0EB7EC02F000019C
:105910001EEF31F035EC31F0F1C233F3F1510301F8
:105920001C6FAA6A4E0EA96E1C51B7EC02F0000162
:105930001EEF31F035EC31F0F1C234F3010E03010A
:10594000345D00010DE1AA6A4F0EA96E310EB7EC6D
:1059500002F0AA6A500EA96EFF0EB7EC02F024D036
:10596000020E0301345D00010DE1AA6A4F0EA96E1B
:10597000320EB7EC02F0AA6A500EA96EFF0EB7EC19
:1059800002F012D0AA6A4F0EA96E310EB7EC02F0E7
:10599000AA6A500EA96E350EB7EC02F0AA6A510E33
:1059A000A96EFF0EB7EC02F01EEF31F035EC31F0CE
:1059B000F1C235F30201C06B0F0E0201C05D0001A0
:1059C0001AE200EEF1F00201C051EB5003011C6F2E
:1059D0000D0E1C5D00010FE0AA6A6E0E0201C025CB
:1059E000A96ED8B0AA2A03011C51B7EC02F002013B
:1059F000C02B0001E1E3AA6A6E0E0201C025A96E68
:105A0000D8B0AA2AFF0EB7EC02F000011EEF31F069
:105A1000B9EC30F084EC20F00201C06B0F0E0201F3
:105A2000C05D00011AE200EEF1F00201C051EB503E
:105A300003011C6F0D0E1C5D00010FE0AA6A100E21
:105A40000201C025A96ED8B0AA2A03011C51B7ECE7
:105A500002F00201C02B0001E1E3AA6A100E02016C
:105A6000C025A96ED8B0AA2AFF0EB7EC02F000013B
:105A70001EEF31F0B9EC30F084EC20F00201C06B85
:105A80000F0E0201C05D000116E200EEF1F002010E
:105A9000C051EB5003011C6F0D0E1C5D00010BE0AB
:105AA000AA6AC0C2A9FF03011C51B7EC02F00201AF
:105AB000C02B0001E5E3AA6AC0C2A9FFFF0EB7EC44
:105AC00002F01EEF31F035EC31F0F1C23FF303018B
:105AD0001E6B1D6B03011E5300011FE10F0E03011E
:105AE0001D5D00011AE200EEF1F003011D51EB50C3
:105AF0001C6F0D0E1C5D000110E05E0E03011D25E4
:105B0000A96E000E1E21AA6E1C51B7EC02F0030113
:105B10001D2B000E1E230001DDE35E0E03011D257B
:105B2000A96E000E1E21AA6EFF0EB7EC02F03F51C7
:105B30003BEC08F0C4EC04F034C02AF033C029F088
:105B400032C028F031C027F0346A336A200E326E3A
:105B5000820E316E2AC038F029C037F028C036F0E6
:105B600027C035F094EC07F034C024F333C023F39E
:105B700032C022F331C021F324C334F023C333F005
:105B800022C332F021C331F094EC06F01C6F150EE5
:105B90001C5D000103E3140E03011C6F03011C5183
:105BA000040D1508000114E3F86A360EF324F66EAE
:105BB0001D0EF420F76E0900F5CF10F00900F5CFA7
:105BC00011F00900F550090054EC03F010C0EBF29D
:105BD00014EC1DF01EEF31F002EC3CF0160EF76EE7
:105BE0000E0EF66E20EC02F0016A030139519DECB5
:105BF00000F00D0E28EC02F000011EEF31F00D0E4A
:105C000028EC02F0160EF76E180EF66E20EC02F07D
:105C1000016A086A196A040E186EA7EC00F02E0ECD
:105C200028EC02F0010E086E2D0EA5EC00F00D0E12
:105C300028EC02F01EEF31F04F0E28EC02F04B0E74
:105C400028EC02F00D0E28EC02F0010E156EF40E99
:105C500034EC03F08DEC31F0BDEF0FF078EC35F063
:105C6000160EF76E2A0EF66E20EC02F0016A16C3CD
:105C700026F015C325F014C324F013C323F0020E3D
:105C8000E1EC00F0560E28EC02F0200E28EC02F0B9
:105C900028EC02F0160EF76E320EF66E20EC02F0D3
:105CA000016A0EC326F00DC325F00CC324F00BC30C
:105CB00023F0010EE1EC00F0430E28EC02F00D0E93
:105CC00028EC02F01EEF31F0140EF76E680EF66E3F
:105CD00020EC02F00D0E28EC02F0939A8A8ADEEC9A
:105CE0001CF04FEC1DF00B0E096EB80E026EFBECB3
:105CF00001F0F9E303011C6F440E1C5D010ED8A4F2
:105D0000000E3A6E640E1C5D010ED8A4000E3A120D
:105D1000000114E00201EB510001E8BE06D00201CF
:105D2000EB53000102E00201EB070001016A0201EE
:105D3000EB51A4EC00F00D0E28EC02F0550E03011F
:105D40001C5D010ED8A4000E3A6E750E1C5D010E8E
:105D5000D8A4000E3A12000112E00201EBBF04D0F9
:105D60007F0EEB5D000102E20201EB2B0001016AF4
:105D70000201EB51A4EC00F00D0E28EC02F0450EF0
:105D800003011C5D010ED8A4000E3A6E650E1C5D69
:105D9000010ED8A4000E3A12000103E03BEC1DF006
:105DA0004DD2530E03011C5D010ED8A4000E3A6EB5
:105DB000730E1C5D010ED8A4000E3A1200010BE018
:105DC0003BEC1DF0AA6A5E0EA96E0201EB51B7EC26
:105DD00002F0000133D214EC1DF085D7CAD984EC4F
:105DE00020F003012A910001F1510C6E4F0E0C5C62
:105DF000010ED8A4000E3A6EF2510C6E4E0E0C5CE1
:105E0000010ED8A4000E3A1604E003012A83000113
:105E100052D0F1510C6E590E0C5C010ED8A4000E3C
:105E20003A6EF2510C6E450E0C5C010ED8A4000EB9
:105E30003A16F3510C6E530E0C5C010ED8A4000EF2
:105E40003A1604E003012A83000135D0F1510C6EAB
:105E50004F0E0C5C010ED8A4000E3A6EF2510C6E7F
:105E6000460E0C5C010ED8A4000E3A16F3510C6ECF
:105E7000460E0C5C010ED8A4000E3A1604E0030195
:105E80002A93000118D0F1510C6E4E0E0C5C010EDD
:105E9000D8A4000E3A6EF2510C6E4F0E0C5C010E3F
:105EA000D8A4000E3A1604E003012A93000102D0A0
:105EB00003012A81000112000D0E28EC02F0160EDB
:105EC000F76E3A0EF66E20EC02F00D0E28EC02F0A2
:105ED0000D0E28EC02F0160EF76E540EF66E20EC46
:105EE00002F00D0E28EC02F0160EF76E720EF66E32
:105EF00020EC02F00D0E28EC02F0160EF76E920E5A
:105F0000F66E20EC02F00D0E28EC02F0160EF76E85
:105F1000AA0EF66E20EC02F00D0E28EC02F0160E22
:105F2000F76EC40EF66E20EC02F00D0E28EC02F0B7
:105F3000160EF76EE80EF66E20EC02F00D0E28EC51
:105F400002F0170EF76E2A0EF66E20EC02F00D0E20
:105F500028EC02F0170EF76E480EF66E20EC02F0F9
:105F60000D0E28EC02F0170EF76E7E0EF66E20EC8A
:105F700002F00D0E28EC02F0170EF76E980EF66E7A
:105F800020EC02F00D0E28EC02F0170EF76EC00E9A
:105F9000F66E20EC02F00D0E28EC02F0170EF76EF4
:105FA000DC0EF66E20EC02F00D0E28EC02F0180E5E
:105FB000F76E020EF66E20EC02F00D0E28EC02F0E9
:105FC000180EF76E300EF66E20EC02F00D0E28EC77
:105FD00002F0180EF76E560EF66E20EC02F00D0E63
:105FE00028EC02F0180EF76E860EF66E20EC02F02A
:105FF0000D0E28EC02F0180EF76EB20EF66E20ECC5
:1060000002F00D0E28EC02F0180EF76EE80EF66E98
:1060100020EC02F00D0E28EC02F0190EF76E140EB3
:10602000F66E20EC02F00D0E28EC02F0190EF76E61
:106030003E0EF66E20EC02F00D0E28EC02F0190E6A
:10604000F76E680EF66E20EC02F00D0E28EC02F0F2
:10605000190EF76EA80EF66E20EC02F00D0E28EC6D
:1060600002F0190EF76ECE0EF66E20EC02F00D0E59
:1060700028EC02F0190EF76EF60EF66E20EC02F028
:106080000D0E28EC02F01A0EF76E1C0EF66E20ECC8
:1060900002F00D0E28EC02F01A0EF76E3E0EF66EB0
:1060A00020EC02F00D0E28EC02F01A0EF76E6A0ECC
:1060B000F66E20EC02F00D0E28EC02F01A0EF76ED0
:1060C0009A0EF66E20EC02F00D0E28EC02F01A0E7D
:1060D000F76ECA0EF66E20EC02F00D0E28EC02F000
:1060E0001A0EF76EF00EF66E20EC02F00D0E28EC94
:1060F00002F01B0EF76E300EF66E20EC02F00D0E65
:1061000028EC02F01B0EF76E660EF66E20EC02F025
:106110000D0E28EC02F01B0EF76EA60EF66E20ECAC
:1061200002F00D0E28EC02F01B0EF76EE00EF66E7C
:1061300020EC02F00D0E28EC02F01C0EF76E000EA3
:10614000F66E20EC02F00D0E28EC02F01C0EF76E3D
:10615000260EF66E20EC02F00D0E28EC02F01C0E5E
:10616000F76E400EF66E20EC02F00D0E28EC02F0F9
:1061700065D003012A950201C06B000100EEF1F029
:106180000201C051EB500C6E200E0C5CD8A4010E25
:106190003A6EFD0EC05D010ED8B0000E3A16000139
:1061A00012E000EEF1F00201C051EB500C6E0D0E4A
:1061B0000C5C000104E103012A85000112000201C8
:1061C000C02B0001DAD70201C02BC051FF080B6EB3
:1061D000CD6B0201CD510B5C000110E30201CD51EA
:1061E000C02500EEF1F0EBCF0CF000EEF1F0CD5158
:1061F0000CC0EBFF0201CD2B0001EBE31200450EBA
:1062000028EC02F0520E28EC02F028EC02F04F0EBF
:1062100028EC02F0520E28EC02F00D0E28EC02F0F1
:10622000630E28EC02F06D0E28EC02F0640E28ECF0
:1062300002F03E0E28EC02F013EF20F04F0E28EC97
:1062400002F04B0E28EC02F00D0E28EC02F0630E6B
:1062500028EC02F06D0E28EC02F0640E28EC02F03F
:106260003E0E28EC02F013EF20F083DF010E020156
:10627000C06F0001F1510C6E0F0B0201F46BF36B58
:10628000F26BF16F000100EEF1F00201C051EB5032
:106290000C6E0D0E0C5C0001D8B43ED0266A256A47
:1062A000246A0A0E236E26C013F025C012F024C003
:1062B00011F023C010F0F4C21BF0F3C21AF0F2C2C6
:1062C00019F0F1C218F053EC04F013C026F012C01C
:1062D00025F011C024F010C023F000EEF1F002010F
:1062E000C051EB500C6E2A6A296A286A0CC027F04C
:1062F0000F0E27142A6A296A286A276E2324F16F51
:1063000028502420F26F29502520F36F2A50262090
:10631000F46FC02B0001B6D7120003011E6B1D6B7A
:106320001EC3AAFF1DC3A9FFB0EC02F01C6F03013E
:106330001C29000112E002EE77F003011D511CC37D
:10634000EBFF1D2B000E1E231EC3AAFF1DC3A9FFBA
:10635000B0EC02F01C6F0001EAD7F36A02EE77F0AE
:1063600003011D51F3CFEBFF1E0EAEEC02F01C6FCC
:106370001C2900010BE1190E0201D36FEA0ED26F46
:10638000850ED16F800ED06F000182D00201D36BD9
:10639000D26BD16BD06BC06B03011C290001D8B448
:1063A00043D0266A256A246A0A0E236E26C013F09B
:1063B00025C012F024C011F023C010F0D3C21BF08E
:1063C000D2C21AF0D1C219F0D0C218F053EC04F0C6
:1063D00013C026F012C025F011C024F010C023F025
:1063E0002A6A296A286A1CC327F00F0E27142A6A12
:1063F000296A286A276E23240201D06F285024209E
:10640000D16F29502520D26F2A502620D36FC02B60
:10641000AA6A1E0EC025A96ED8B0AA2AB0EC02F056
:1064200003011C6F0001B8D7070E0201D35D000104
:1064300014E311E1170E0201D25D00010EE30BE13E
:10644000CB0E0201D15D000108E305E1C00E02019F
:10645000D05D000102E3000E01D0010E3A6E810E04
:106460000201D05DD90ED1599F0ED259380ED359A1
:10647000000102E2000E01D0010E3A1209E0190EED
:106480000201D36FEA0ED26F850ED16F800ED06FEE
:106490000301306B2F6B2E0EAEEC02F01C6F1C292B
:1064A000000107E1030E0301306F7A0E2F6F000128
:1064B00036D00201C06B03011C29000130E0246AC0
:1064C0000A0E236E24C019F02350186E03012F0307
:1064D000F3CF23F0F4CF24F019502F03F3502426E8
:1064E00018503003F3502426286A1CC327F00F0EDF
:1064F0002716000E2816275023242F6F28502420FB
:10650000306F0201C02BAA6A2E0EC025A96ED8B02A
:10651000AA2AB0EC02F003011C6F0001CCD70301E2
:10652000326B316B3E0EAEEC02F01C6F1C29000189
:1065300007E1270E0201F86F100EF76F000173D00C
:106540000201C06B03011C29000130E0246A0A0E1D
:10655000236E24C019F02350186E03013103F3CFCA
:1065600023F0F4CF24F019503103F35024261850AF
:106570003203F3502426286A1CC327F00F0E271677
:10658000000E281627502324316F28502420326F04
:106590000201C02BAA6A3E0EC025A96ED8B0AA2A55
:1065A000B0EC02F003011C6F0001CCD703013253A1
:1065B000000109E12D0E0301315D000104E2030138
:1065C000326B2D0E316F050E0301325D00010BE3BE
:1065D00005E1DD0E0301315D000105E3050E030158
:1065E000326FDC0E316F030131512D0A321100017F
:1065F00007E1560E0201F86FCE0EF76F000113D0BF
:10660000136A0F0E126E420E116E400E106E31C3E1
:1066100018F032C319F01A6A1B6AD3EC03F011C0E8
:10662000F8F210C0F7F24E0EAEEC02F00301336F39
:106630003329000105E1070E0301336F000103D088
:106640000F0E03013317070E0301335DD8A4010EAB
:106650003A6E080E335DD8A4010E3A16000103E02D
:10666000080E0301336F0001AA6A4F0EA96EB0EC49
:1066700002F003011C6F1C29000108E1D8900201FF
:10668000F735F96FF835FA6F000166D00F0E030188
:106690001C150201C06FAA6A500EA96EB0EC02F080
:1066A00003011C6F1C29000119E0246A0A0E236EE5
:1066B00024C010F00201C0512302F3CF23F0F4CF25
:1066C00024F01002F3502426286A1CC327F00F0E72
:1066D0002716000E281623502724C06F010E020132
:1066E000C05DD8A4010E3A6E020EC05DD8A4010EA2
:1066F0003A160F0EC05DD8A4010E3A16000103E051
:10670000010E0201C06F0001C0C234F30F0E02017E
:10671000C05D000116E1F7C231F0F8C232F03DEC85
:1067200008F0386A376A400E366E7F0E356E94EC8C
:1067300007F0E2EC07F00201F96F32C0FAF2000153
:106740000AD00201C051F703F3CFF9F2F4CFFAF205
:10675000F803F350FA2700015E0EAEEC02F00301DD
:106760001C6F1C29000105E10A0E03013F6F0001A7
:106770002FD003013F6B0201C06B03011C290001F4
:1067800027E0246A0A0E236E24C010F003013F5153
:106790002302F3CF23F0F4CF24F01002F350242689
:1067A000286A1CC327F00F0E2716000E2816235048
:1067B00027243F6F0201C02BAA6A5E0EC025A96E76
:1067C000D8B0AA2AB0EC02F003011C6F0001D5D7A3
:1067D00003013F513BEC08F0C4EC04F034C02AF054
:1067E00033C029F032C028F031C027F0346A336A50
:1067F000200E326E820E316E2AC038F029C037F07A
:1068000028C036F027C035F094EC07F034C024F3EC
:1068100033C023F332C022F331C021F324C334F058
:1068200023C333F022C332F021C331F094EC06F0DD
:106830001C6F150E1C5D000103E3140E03011C6F99
:1068400003011C51040D1508000114E3F86A8E0EB3
:10685000F324F66E1D0EF420F76E0900F5CF10F04C
:106860000900F5CF11F00900F550090054EC03F0D0
:1068700010C0EBF2030E03011C27150E1C5D000176
:1068800003E3140E03011C6F03011C51040D1508D2
:10689000000114E3F86AE60EF324F66E1D0EF420F0
:1068A000F76E0900F5CF10F00900F5CF11F00900DF
:1068B000F550090054EC03F010C036F33C0E030110
:1068C000286F6E0EAEEC02F01C6F1C290001D8B4CC
:1068D0004BD00201C06B0301356B03011C29000181
:1068E00027E0246A0A0E236E24C010F003013551FC
:1068F0002302F3CF23F0F4CF24F01002F350242628
:10690000286A1CC327F00F0E2716000E28162350E6
:106910002724356F0201C02BAA6A6E0EC025A96E0E
:10692000D8B0AA2AB0EC02F003011C6F0001D5D741
:10693000140E0301355D000103E2140E0301356FEF
:10694000790E0301355D000103E3780E0301356F15
:106950000001040E116EB00E106E156A35C314F0EE
:1069600001EC04F00301286F0001810EAEEC02F08F
:106970000201D46FB0EC02F0D56FB0EC02F0D66F2C
:10698000B0EC02F0D76F000ED75D000114E311E107
:10699000980E0201D65D00010EE30BE1960E020196
:1069A000D55D000108E305E1800E0201D45D000120
:1069B00002E3000E01D0010E3A6E410E0201D45DD9
:1069C0008A0ED559F70ED659010ED759000102E2A9
:1069D000000E01D0010E3A1209E0010E0201D76F3C
:1069E000C90ED66FC30ED56F800ED46F0001850E11
:1069F000AEEC02F00201D86FB0EC02F0D96FD9AF63
:106A000006D0D00ED85D8A0ED959000102E3000EDF
:106A100001D0010E3A6E0201D9BF0AD0750ED95DC0
:106A200007E3000107E1310E0201D85D000102E237
:106A3000000E01D0010E3A12000105E0040E020121
:106A4000D96FB00ED86F0001800EAEEC02F00301DA
:106A50003E6F7E0EAEEC02F03C6F7F0EAEEC02F0AD
:106A60003D6F870EAEEC02F0406F880EAEEC02F088
:106A70000201EC6F890EAEEC02F09B6E03012A97C7
:106A8000296B01EEDEF0EF6A01EEEEF0EF6A01EE47
:106A9000FEF0EF6A300E0201BB6F02EE3EF0EF6ACD
:106AA00003013A6B02EE0EF0EE6E2E0EEE6E300E1D
:106AB000EE6EEF6A02EE1EF0EF6A02EE2EF0EF6A63
:106AC0000201FC6BFB6B9BCF39F30301D89239BBFE
:106AD000D882D8B2398DD8A2399DD89239BBD88204
:106AE000D8B2398FD8A2399F960E2E6F00011200AE
:106AF000010E0201896F8A6F080E8B6F00017BEC1B
:106B000041F01C0EF76E640EF66E20EC02F0016A86
:106B100002018951A4EC00F00D0E28EC02F01C0ECD
:106B2000F76E740EF66E20EC02F0016A020E086E2B
:106B30008A5188EC00F0020E086E8B5188EC00F050
:106B40000D0E28EC02F01C0EF76E7E0EF66E20EC99
:106B500002F0016A020E086E8C5188EC00F00D0EF6
:106B600028EC02F01C0EF76E8E0EF66E20EC02F092
:106B7000016A020E086E8D5188EC00F0020E086E5C
:106B80008E5188EC00F00D0E28EC02F01C0EF76E12
:106B9000A20EF66E20EC02F0016A020E086E8F5112
:106BA00088EC00F00D0E28EC02F01C0EF76EB20E11
:106BB000F66E20EC02F0016A020E086E905188EC2D
:106BC00000F00D0E28EC02F0030E0201896F140E86
:106BD0008A6F180E8B6F8C6B060E8D6F00017BEC2D
:106BE00041F002018B5103011E6F02018C51030120
:106BF0001D6F1DC331F01EC332F03DEC08F0386A42
:106C0000376A400E366E800E356E94EC07F034C055
:106C100026F033C025F032C024F031C023F0386AAA
:106C2000376A200E366E890E356E26C034F025C0C8
:106C300033F024C032F023C031F02EEC07F034C022
:106C400016F333C015F332C014F331C013F302014D
:106C50008D5103011E6F02018E5103011D6F246BC4
:106C6000C00E236F600E226F7C0E216F1DC331F0AA
:106C70001EC332F03DEC08F024C338F023C337F0D4
:106C800022C336F021C335F094EC07F034C026F06F
:106C900033C025F032C024F031C023F0386A800EB2
:106CA000376E120E366E870E356E26C034F025C054
:106CB00033F024C032F023C031F09EEC06F034C033
:106CC0000EF333C00DF332C00CF331C00BF30001EF
:106CD00012000301206B1F6B0201C06B0A0E020140
:106CE000C05D00010FE2010EC6EC02F00C6E24C084
:106CF0000DF00C5003011F270D5020230201C02B63
:106D00000001ECE31FC331F020C332F03DEC08F08A
:106D1000386A400E376E1C0E366E8A0E356E9EEC4B
:106D200006F034C026F033C025F032C024F031C064
:106D300023F0386A376A480E366E840E356E26C0E8
:106D400034F025C033F024C032F023C031F02EECF3
:106D500007F034C00AF333C009F332C008F331C07E
:106D600007F312000301206B1F6B0201C06B0A0EB8
:106D70000201C05D00010FE2000EC6EC02F00C6ED5
:106D800024C00DF00C5003011F270D5020230201D9
:106D9000C02B0001ECE31FC331F020C332F03DEC07
:106DA00008F0386A400E376E1C0E366E8A0E356E4D
:106DB0009EEC06F034C026F033C025F032C024F03B
:106DC00031C023F0386A376A480E366E840E356E4D
:106DD00026C034F025C033F024C032F023C031F097
:106DE0002EEC07F034C012F333C011F332C010F3AD
:106DF00031C00FF312000301206B1F6B0201C06B47
:106E00000A0E0201C05D00010FE2030EC6EC02F0A3
:106E10000C6E24C00DF00C5003011F270D502023D1
:106E20000201C02B0001ECE3386A400E376E1C0EE5
:106E3000366E8B0E356E20C332F01FC331F03DEC41
:106E400008F02EEC07F034C000F333C0FFF232C07C
:106E5000FEF231C0FDF212000301206B1F6B020134
:106E6000C06B0A0E0201C05D00010FE20F0EC6ECFE
:106E700002F00C6E24C00DF00C5003011F270D50C2
:106E800020230201C02B0001ECE3386A400E376E6C
:106E90001C0E366E8B0E356E20C332F01FC331F0E0
:106EA0003DEC08F02EEC07F034C004F333C003F3DC
:106EB00032C002F331C001F312000301206B1F6BDB
:106EC0001E6B1D6B0201C06B0A0E0201C05D00014A
:106ED00019E2040EC6EC02F00C6E24C00DF00C504A
:106EE00003011F270D5020230F0EC6EC02F00C6E7D
:106EF00024C00DF00C501D270D501E230201C02B85
:106F00000001E2E3386A400E376E1C0E366E8B0EBF
:106F1000356E1EC332F01DC331F03DEC08F02EEC8F
:106F200007F034C004F333C003F332C002F331C0BE
:106F300001F303011F511D5D056F20511E59066F9E
:106F400006C31FF005C31EF0196A050E186E18EC73
:106F500004F0056F11C006F300011200D76AD66A6B
:106F600003011E6B1D6B2A8382A02A93320E33EC21
:106F700003F00001E86A03012AB3010F82B001089F
:106F800000012CE103011D2B000E1E23320E33ECF9
:106F900003F0020E1E5D000120E305E1590E03011E
:106FA0001D5D00011AE301EE47F00D0EEE6E0A0EB4
:106FB000EE6E1C0EF76EBE0EF66EB3EC04F00D0E08
:106FC000EE6E0A0EEE6EEF6A000178EC1EF0270EF0
:106FD000156E100E34EC03F0C1D7CBD782B0FED7BC
:106FE00082A0FED7D58E82B0FED782A0FED7D59ED6
:106FF000D6CF18F3D7CF19F3F40E0301195DBA0EEB
:10700000D8B4185D000102E20301392BF50E03012B
:10701000195D000108E305E11F0E0301185D000181
:1070200002E3030139073F0E030139159B6EF40E8D
:10703000195DBA0ED8B4185D000102E2000E01D04D
:10704000010E3A6EF50E0301195D000108E305E13A
:107050001F0E0301185D000102E3000E01D0010EB6
:107060003A16000106E0AA6A890EA96E9B50B7EF96
:1070700002F001EE47F0200EEE6EEE6E020E016E93
:10708000086A19C319F018C318F0A7EC00F0200E15
:10709000EE6EEE6E020E016E030139519DEC00F0B2
:1070A0000D0EEE6EEF6A000178EC1EF0030E156E09
:1070B000E80E34EC03F0D76AD66A90D7949A8B8A9C
:1070C00003013D3500011CE2800E026E400E096E88
:1070D000216A40C320F0066A056A200E016E120E76
:1070E000F76E1C0EF66E0900F55003E0B3EC01F0EC
:1070F000FAD70D0EB3EC01F00A0EB3EC01F03BD061
:10710000800E026E400E096E216A40C320F0066AAE
:10711000056A200E016EB50EB3EC01F0620EB3EC01
:1071200001F0060EB3EC01F0570EB3EC01F0080EBF
:10713000B3EC01F0000EB3EC01F0010EB3EC01F082
:10714000000EB3EC01F0000EB3EC01F0000EB3EC56
:1071500001F0500EB3EC01F04F0EB3EC01F0540E01
:10716000B3EC01F0530EB3EC01F0AC0EB3EC01F054
:10717000850EB3EC01F0A1DE1C0EF76ED40EF66E98
:1071800020EC02F0016A086A06C319F005C318F082
:10719000A7EC00F0130E156E880E34EC03F0949AF1
:1071A0008B9A03013D3500011CE2800E026E400EF9
:1071B000096E216A40C320F0066A056A200E016E3E
:1071C000120EF76E2A0EF66E0900F55003E0B3ECCE
:1071D00001F0FAD70D0EB3EC01F00A0EB3EC01F09A
:1071E0003BD0800E026E400E096E216A40C320F033
:1071F000066A056A200E016EB50EB3EC01F0620E50
:10720000B3EC01F0060EB3EC01F0570EB3EC01F055
:10721000080EB3EC01F0000EB3EC01F0010EB3EC7C
:1072200001F0000EB3EC01F0000EB3EC01F0000E23
:10723000B3EC01F0200EB3EC01F04E0EB3EC01F014
:10724000550EB3EC01F0520EB3EC01F07B0EB3EC33
:1072500001F0C30EB3EC01F030DE1C0EF76EE20E4F
:10726000F66E20EC02F0016A086A06C319F005C345
:1072700018F0A7EC00F00D0E28EC02F0130E156EBE
:10728000880E34EC03F0096A010E026EFBEC01F08B
:10729000D8A014D703011C6F450E1C5D010ED8A4A5
:1072A000000E3A6E650E1C5D010ED8A4000E3A1257
:1072B000000104E03AEC1FF01EEF31F0FFD640C3AE
:1072C00025F300EEF1F0240EEE6E470EEE6EEF6A3F
:1072D000800E026E800E096E216A40C320F00B0EF4
:1072E000066EB80E056E72EC01F0D8A0CBD0240863
:1072F000FAE172EC01F0D8A0C5D003011C6F020EB8
:107300000201C06F510E0201C05D00011AE2800E41
:10731000026E800E096E216A40C320F08FEC01F0EE
:1073200003011C6F00EEF1F00201C0511CC3EBFF22
:107330000D0E03011C5D000104E00201C02B0001E1
:10734000E1E30201C029F10FE96E000EEA6AEA22C8
:10735000EF6ACD6B0201CD51C05D00010BE300EE81
:10736000F1F00201CD51EB5028EC02F00201CD2BDF
:107370000001F0E3030E096EE80E026EFBEC01F073
:10738000D8A09DD703011C6F550E1C5D010ED8A41B
:10739000000E3A6E750E1C5D010ED8A4000E3A1256
:1073A000000109E00301402B016A4051A4EC00F008
:1073B0000D0E28EC02F0440E03011C5D010ED8A452
:1073C000000E3A6E640E1C5D010ED8A4000E3A1237
:1073D000000109E003014007016A4051A4EC00F0FC
:1073E0000D0E28EC02F0530E03011C5D010ED8A413
:1073F000000E3A6E730E1C5D010ED8A4000E3A12F8
:1074000000011AE0AA6A870EA96E03014051B7EC89
:1074100002F00D0E28EC02F01C0EF76EF40EF66E64
:1074200020EC02F0016A4051A4EC00F00D0E28ECB3
:1074300002F000011EEF31F0450E03011C5D010E4C
:10744000D8A4000E3A6E650E1C5D010ED8A4000E85
:107450003A12000116E025C340F30D0E28EC02F0AD
:107460001C0EF76EFC0EF66E20EC02F0016A0301B2
:107470004051A4EC00F00D0E28EC02F000011EEFCC
:1074800031F01FD71D0EF76E180EF66E20EC02F0CD
:1074900071D769EC36F0FBEC36F05EEC1DF0E4ECF5
:1074A00035F001EE47F0240EEE6EEE6EEE6EEE6EEF
:1074B00012EE77F0110EE75204E0E6CFEEFFE82E71
:1074C000FAD72C0EEE6E020E016E0EC326F00DC31F
:1074D00025F00CC324F00BC323F0010EE1EC00F007
:1074E0002C0EEE6E020E016E0AC326F009C325F0C3
:1074F00008C324F007C323F0010EE1EC00F02C0ECA
:10750000EE6E020E016E16C326F015C325F014C3ED
:1075100024F013C323F0E1EC00F02C0EEE6E020E0B
:10752000016E00C326F0FFC225F0FEC224F0FDC2AA
:1075300023F0E1EC00F0EF6A03011B6B01EE47F072
:10754000E86AEE5202E0E83EFCD70B6E040E020140
:10755000CD6F0201CD510B5C00010FE301EE47F04E
:107560000201CD51E926000EEA22EF500C6E030114
:107570001B1B0201CD2B0001ECE301EE47F0EE50A6
:10758000FEE1ED522A0EEE6E020E016E086E030150
:107590001B5188EC00F00D0EEE6E0A0EEE6EEF6AD7
:1075A000000178EC1EF0130E096E880E026EFBECE3
:1075B00001F0D8A06ED703011C6F450E1C5D010EB3
:1075C000D8A4000E3A6E650E1C5D010ED8A4000E04
:1075D0003A120001D8A41EEF31F05BD722EC1EF066
:1075E000016A086ADFC226F0DEC225F0DDC224F09F
:1075F000DCC223F03FEC01F00D0E28EC02F068EC49
:107600001DF0020E0201896F220E8A6F8B6B080E2D
:107610008C6F00017BEC41F01D0EF76E2E0EF66EA6
:1076200020EC02F0016A02018B51A4EC00F0200E64
:1076300028EC02F08C51A4EC00F0200E28EC02F0B3
:107640008D51A4EC00F0200E28EC02F08E51A4EC39
:1076500000F00D0E28EC02F0030E096EE80E026E2B
:10766000FBEC01F00001CDE303011C6F450E1C5D36
:10767000010ED8A4000E3A6E650E1C5D010ED8A452
:10768000000E3A120001D8A41EEF31F0BAD7949E32
:107690008B9E810E026E010E096E810E036E040E2A
:1076A000046E010E0A6E120E106E08EC03F0400E0E
:1076B000106E08EC03F0080E106E08EC03F0106A70
:1076C00008EC03F0949E8B8E81A6FED7949E8B9E31
:1076D000810E026E010E096E810E036E040E046EA1
:1076E000010E0A6E440E106E08EC03F0810E026E5D
:1076F000020E096E810E036E040E046E0A6ADCEC43
:1077000002F010C01CF303011C29000108E0949E44
:107710008B8E010E33EC03F0949E8B9ED9D7810E95
:10772000026E020E096E810E036E040E046E0A6A6A
:10773000DCEC02F010C041F3DCEC02F010C042F3CC
:10774000DCEC02F010C043F3DCEC02F010C044F3B8
:10775000DCEC02F010C045F3DCEC02F010C046F3A4
:10776000DCEC02F010C047F3DCEC02F010C048F390
:10777000949E8B8E016A020E086E0301415188ECC3
:1077800000F0200E28EC02F0020E086E425188EC48
:1077900000F0200E28EC02F0020E086E435188EC37
:1077A00000F0200E28EC02F0020E086E445188EC26
:1077B00000F0200E28EC02F0020E086E455188EC15
:1077C00000F0200E28EC02F0020E086E465188EC04
:1077D00000F0200E28EC02F0020E086E475188ECF3
:1077E00000F0200E28EC02F0020E086E485188ECE2
:1077F00000F0200E28EC02F00D0E28EC02F0000143
:107800001EEF31F0D76AD66A82B0FED782A0FED7CB
:10781000D58E82B0FED782A0FED7D59ED6CF18F3E4
:10782000D7CF19F3F40E0301195D000106E307E158
:10783000A70E0301185D000102E20301392BF50ECA
:107840000301195D000108E305E13C0E0301185D29
:10785000000102E303013907F40E0301195D000181
:1078600006E307E1A70E0301185D000102E2000E26
:1078700001D0010E3A6EF50E0301195D000108E317
:1078800005E13C0E0301185D000102E3000E01D08A
:10789000010E3A160001D8A412003F0E030139155B
:1078A0009B6E140E33EC03F00001ACD70201CD6BDC
:1078B0000001DFEC1EF0246A0A0E236E020144511F
:1078C0000C6E286A0CC027F00F0E2716000E281623
:1078D00024C019F02350186E2702F3CF23F0F4CF01
:1078E00024F019502702F350242618502802F35090
:1078F000242645510E6E286A0EC027F00F0E27165B
:10790000000E2816235027240301516F246A0A0E03
:10791000236E020146510C6E286A0CC027F00F0E30
:107920002716000E281624C019F02350186E2702BF
:10793000F3CF23F0F4CF24F019502702F35024267C
:1079400018502802F350242647510E6E286A0EC0A4
:1079500027F00F0E2716000E2816235027240301A8
:10796000526F386A376A700E366E840E356E525119
:107970003BEC08F02EEC07F034C026F033C025F0C5
:1079800032C024F031C023F051513BEC08F026C046
:1079900038F025C037F024C036F023C035F0A0EC15
:1079A00006F034C024F333C023F332C022F331C0D5
:1079B00021F3246A0A0E236E020149510C6E286AD3
:1079C0000CC027F00F0E2716000E281624C019F041
:1079D0002350186E2702F3CF23F0F4CF24F0195070
:1079E0002702F350242618502802F35024264A5127
:1079F0000E6E286A0EC027F00F0E2716000E2816EE
:107A0000235027240301566F0201CD6B0001DEECE9
:107A10001EF002EE44F0EECFF3FFEFCFF4FFF35091
:107A20004E0AF41005E15A0E03015127000115D04A
:107A3000030151515A08516F525300010EE00301E6
:107A4000510752513C08526F5653000105E00301A3
:107A5000520756516408566F0001D89003015237FF
:107A6000D89056370201CD6B0001DDEC1EF0246A80
:107A7000640E236E020144510C6E286A0CC027F07C
:107A80000F0E2716000E281624C019F02350186E6A
:107A90002702F3CF23F0F4CF24F019502702F3503C
:107AA000242618502802F3502426286A0A0E276E2E
:107AB00045510E6E2C6A0EC02BF00F0E2B16000EC9
:107AC0002C1628C019F02750186E2B02F3CF27F080
:107AD000F4CF28F019502B02F350282618502C020E
:107AE000F3502826275023262850242246510F6E73
:107AF000286A0FC027F00F0E2716000E28162750F1
:107B000023240301536F28502420546F246A0A0E43
:107B1000236E020147510C6E286A0CC027F00F0E2D
:107B20002716000E281624C019F02350186E2702BD
:107B3000F3CF23F0F4CF24F019502702F35024267A
:107B400018502802F350242648510E6E286A0EC0A1
:107B500027F00F0E2716000E2816235027240301A6
:107B6000556F386A376A700E366E840E356E555111
:107B70003BEC08F02EEC07F034C026F033C025F0C3
:107B800032C024F031C023F053C331F054C332F07B
:107B90003DEC08F026C038F025C037F024C036F0A0
:107BA00023C035F0A0EC06F034C024F333C023F337
:107BB00032C022F331C021F3246A0A0E236E02017F
:107BC0004A510C6E286A0CC027F00F0E2716000EC3
:107BD000281624C019F02350186E2702F3CF23F083
:107BE000F4CF24F019502702F3502426185028020D
:107BF000F35024264B510E6E286A0EC027F00F0E4C
:107C00002716000E2816235027240301576F020160
:107C1000CD6B0001DCEC1EF002EE44F0EECFF3FF82
:107C2000EFCFF4FFF350450AF41007E1B40E03015F
:107C30005327000E542300011AD003015351B408F6
:107C4000536F000E5455546F5553000110E003015B
:107C50005307000E545B55513C08556F57530001B4
:107C600005E00301550757516408576F000102EE04
:107C700044F0EF6A54C311F053C310F0156A140EA8
:107C8000146E01EC04F0236E11C024F0410E232485
:107C900003011C6F02EE44F0EE50FEE1ED521CC3F6
:107CA000EEFFEF6A51C310F00A0EFEEC03F0236EF4
:107CB000246A410E23241C6F02EE44F0EE50FEE1D4
:107CC000ED521CC3EEFFEF6A246A300E236E54C3DC
:107CD00028F053C327F028C011F027C010F0156A10
:107CE000140E146E01EC04F019C028F018C027F02F
:107CF000D89028322732235027241C6F02EE44F0FC
:107D0000EE50FEE1ED521CC3EEFFEF6A116A51C363
:107D100010F0156A0A0E146E01EC04F019C024F07C
:107D200018C023F0300E23241C6F02EE44F0EE50F6
:107D3000FEE1ED521CC3EEFFEF6A246A410E236E92
:107D4000000E53B1010E286A276E28503C0DF3CF68
:107D500028F027503C0DF3CF27F0F450282655513A
:107D60002726000E282228C011F027C010F0156A1F
:107D7000050E146E01EC04F0276E11C028F023509C
:107D800027241C6F02EE44F0EE50FEE1ED521CC3BE
:107D9000EEFFEF6A52C310F0050EFEEC03F0236E07
:107DA000246A410E23241C6F02EE44F0EE50FEE1E3
:107DB000ED521CC3EEFFEF6A000E3DBB010E3A6EA2
:107DC000000E2AB7010E3A120001D8B4DFD03C0EE3
:107DD000030153A1000E236E53A1000E246E5551D2
:107DE00023241D6F000E24201E6F1EC311F01DC31F
:107DF00010F0156A050E146E01EC04F018C01CF3A7
:107E00001C51640DF3CF23F0F4CF24F057512324F9
:107E10001D6F000E24201E6F1EC311F01DC310F035
:107E2000156A320E146E01EC04F0236E11C024F0BA
:107E3000300E23241C6F02EE44F0EE50FEE1ED52B2
:107E40001CC3EEFFEF6A1EC311F01DC310F0156ACC
:107E5000320E146E01EC04F018C057F3116A52C3CD
:107E600010F0156A050E146E01EC04F018C01CF336
:107E70001C51640DF3CF23F0F4CF24F0565123248A
:107E80001D6F000E24201E6F1EC311F01DC310F0C5
:107E9000156A320E146E01EC04F0236E11C024F04A
:107EA000300E23241C6F1EC311F01DC310F0156A81
:107EB000320E146E01EC04F018C056F302EE44F0DA
:107EC000EE50FEE1ED521CC3EEFFEF6ADF0E386E9E
:107ED0004F0E376E050E366E800E356E57513BECE9
:107EE00008F02EEC07F034C026F033C025F032C085
:107EF00024F031C023F0346A336A020E326E850EEC
:107F0000316E26C038F025C037F024C036F023C0CB
:107F100035F0A0EC06F0E2EC07F01C6F02EE44F046
:107F2000EE50FEE1ED521CC3EEFFEF6ADF0E386E3D
:107F30004F0E376E050E366E800E356E56513BEC89
:107F400008F02EEC07F034C026F033C025F032C024
:107F500024F031C023F0346A336A020E326E850E8B
:107F6000316E26C038F025C037F024C036F023C06B
:107F700035F0A0EC06F0E2EC07F01C6F02EE44F0E6
:107F8000EE50FEE1ED521CC3EEFFEF6A000112005D
:107F900003013D510001E8A601D0120069EC36F062
:107FA000346A336AC00E326E7F0E316E0AC338F007
:107FB00009C337F008C336F007C335F01CEC06F0F0
:107FC0000108D8B46AD00AC338F009C337F008C32F
:107FD00036F007C335F0660E346E336E4E0E326ED9
:107FE000830E316E9EEC06F034C026F033C025F0CF
:107FF00032C024F031C023F0346A336A2A0E326E64
:10800000850E316E26C038F025C037F024C036F01A
:1080100023C035F094EC07F034C024F333C023F3CD
:1080200032C022F331C021F324C334F023C333F030
:1080300022C332F021C331F0386A376A7E0E356EC2
:10804000800E32AE000E366EA0EC06F0E2EC07F0C9
:1080500034BE03D03FEC08F002D041EC08F034C04D
:108060002AF033C029F032C028F031C027F0D9C23D
:1080700032F0D8C231F035EC08F02AC038F029C00F
:1080800037F028C036F027C035F09EEC06F0E2EC61
:1080900007F00201DA6F32C0DBF200010AC334F0EC
:1080A00009C333F008C332F007C331F0386A376AC6
:1080B000C00E366E7F0E356E58EC06F03A6E0AC36F
:1080C00034F009C333F008C332F007C331F0660E51
:1080D000386E376EE60E366E810E356E1CEC06F08D
:1080E0003A1607E0B60E0201D85DDA6F080ED959CC
:1080F000DB6F00010AC334F009C333F008C332F068
:1081000007C331F0660E386E376EE60E366E810E9E
:10811000356E1CEC06F00108D8B4ABD0266A256A8F
:10812000800E246E7F0E236E660E2A6E296E860EDA
:10813000286E810E276E2AC034F029C033F028C083
:1081400032F027C031F00AC338F009C337F008C352
:1081500036F007C335F09EEC06F034C02AF033C089
:1081600029F032C028F031C027F0346A336A4C0E4F
:10817000326E850E316E2AC038F029C037F028C023
:1081800036F027C035F094EC07F034C02AF033C045
:1081900029F032C028F031C027F026C038F025C0C1
:1081A00037F024C036F023C035F02AC034F029C09F
:1081B00033F028C032F027C031F094EC07F034C01F
:1081C00024F333C023F332C022F331C021F3D9C2E8
:1081D00032F0D8C231F035EC08F0386AE00E376E74
:1081E000080E366E8A0E356EA0EC06F034C026F00E
:1081F00033C025F032C024F031C023F024C334F062
:1082000023C333F022C332F021C331F0386A376A16
:108210007E0E356E800E32AE000E366EA0EC06F08D
:10822000E2EC07F034BE03D03FEC08F002D041ECA2
:1082300008F034C02AF033C029F032C028F031C031
:1082400027F026C034F025C033F024C032F023C01C
:1082500031F02AC038F029C037F028C036F027C0E6
:1082600035F09EEC06F0E2EC07F00201DA6F32C066
:10827000DBF20001DBC232F0DAC231F035EC08F09B
:10828000C8C238F0C7C237F0C6C236F0C5C235F032
:1082900094EC07F094EC06F00201EF6F32C0F0F2BC
:1082A0000001ABEF1DF081A6FED7949E8B9E0201CC
:1082B00089510B6E010E0301586F030158510B5C7D
:1082C000000116E3810E026E010E096E810E036E2F
:1082D000040E046E010E0A6E02EE89F0030158517D
:1082E000EB50106E08EC03F00301582B0001E5E39E
:1082F000949E8B8E12008194D6DF81A6FED7949E29
:108300008B9E810E026E010E096E810E036E040EAD
:10831000046E010E0A6E440E106E08EC03F0810E1E
:10832000026E020E096E810E036E040E046E0A6A5E
:10833000DCEC02F010C01CF303011C29000108E072
:10834000949E8B8E010E33EC03F0949E8B9ED9D7B6
:1083500002EE89F003015851EB500C6E0C041C6FB7
:10836000586B030158511C5D000115E3810E026E2C
:10837000020E096E810E036E040E046E0A6ADCECB6
:1083800002F002EE89F00301585110C0EBFF030127
:10839000582B0001E6E3949E8B8E1200010E020121
:1083A000896F8A6F080E8B6F0001A5DF02018B5168
:1083B0000C6E640E0C5C000102E103012A890201CB
:1083C000CF6B020ECE6F03012A510001E8B892D0A4
:1083D0001F0E0201D35D000114E311E14A0E0201F8
:1083E000D25D00010EE30BE1DD0E0201D15D000163
:1083F00008E305E1400E0201D05D000102E3000E3A
:1084000001D0010E3A6E010E0201D05DB10ED159BC
:10841000080ED259190ED359000102E2000E01D004
:10842000010E3A1605E0040E0201CE6F020ECF6F68
:10843000140E0201D35D000114E311E1DC0E020110
:10844000D25D00010EE30BE1930E0201D15D00014C
:1084500008E305E1800E0201D05D000102E3000E99
:1084600001D0010E3A6E010E0201D05D7F0ED1598E
:10847000ED0ED259100ED359000102E2000E01D0C8
:10848000010E3A1605E0060E0201CE6F030ECF6F05
:108490000A0E0201D35D000114E311E16E0E020128
:1084A000D25D00010EE30BE1490E0201D15D000136
:1084B00008E305E1C00E0201D05D000102E3000EF9
:1084C00001D0010E3A6E810E0201D05DBF0ED1596E
:1084D000760ED259080ED359000102E2000E01D0E7
:1084E000010E3A1605E00C0E0201CE6F050ECF6F9D
:1084F000000151D0400E0201D05D720ED159050E1F
:10850000D2592A0ED359000105E2030E0201CE6FA3
:10851000010ECF6FC00E0201D05DEC0ED1594F0E8F
:10852000D2591C0ED359000105E2040E0201CE6F90
:10853000020ECF6F400E0201D05D5A0ED1590A0EC5
:10854000D259150ED359000105E2060E0201CE6F75
:10855000030ECF6FC00E0201D05DD90ED1593E0E71
:10856000D2590E0ED359000105E2080E0201CE6F5A
:10857000040ECF6F400E0201D05DCE0ED1598C0E8D
:10858000D2590A0ED359000105E20C0E0201CE6F3A
:10859000050ECF6F0001136A080E126E116A106A81
:1085A0001B6A1A6A196ACEC218F053EC04F013C0A1
:1085B000F4F212C0F3F211C0F2F210C0F1F2D7C21D
:1085C00034F0D6C233F0D5C232F0D4C231F03FEC31
:1085D00008F034C038F033C037F032C036F031C064
:1085E00035F0F4C234F0F3C233F0F2C232F0F1C22B
:1085F00031F03FEC08F02EEC07F034C0C8F233C085
:10860000C7F232C0C6F231C0C5F2D7C213F0D6C22B
:1086100012F0D5C211F0D4C210F01B6A1A6A196A9E
:10862000CEC218F0D3EC03F013C0BFF212C0BEF2FA
:1086300011C0BDF210C0BCF2D3C213F0D2C212F00E
:10864000D1C211F0D0C210F0BFC21BF0BEC21AF0EE
:10865000BDC219F0BCC218F0D3EC03F013C026F071
:1086600012C025F011C024F010C023F02304020131
:10867000C06FD3C213F0D2C212F0D1C211F0D0C277
:1086800010F0BFC21BF0BEC21AF0BDC219F0BCC2CE
:1086900018F0D3EC03F030C0F4F22FC0F3F22EC088
:1086A000F2F22DC0F1F2BFC234F0BEC233F0BDC24F
:1086B00032F0BCC231F03FEC08F034C038F033C0C7
:1086C00037F032C036F031C035F0F4C234F0F3C2C6
:1086D00033F0F2C232F0F1C231F03FEC08F02EEC90
:1086E00007F034C0C4F233C0C3F232C0C2F231C0AA
:1086F000C1F2346A336A326A7F0E316EC4C238F016
:10870000C3C237F0C2C236F0C1C235F0A0EC06F0E9
:1087100034C0C4F233C0C3F232C0C2F231C0C1F2BD
:10872000346A336A326A920E316EC4C238F0C3C200
:1087300037F0C2C236F0C1C235F094EC07F0E2EC7B
:1087400007F0C96F32C0CAF233C0CBF234C0CCF2EA
:10875000CBC2E2F2CAC2E1F2C9C2E0F2080E896FEE
:10876000110E8A6F400E8B6F040E8C6F8D6BC0C222
:108770008EF2E2C28FF2E1C290F2E0C291F2000109
:1087800053EF41F0719E0301A56BA46BA36BA26B29
:10879000A96BA86BA76BA66BA1EC02F0EE0E6BECBD
:1087A00002F0AA0E6BEC02F04FEC02F05B6F4FECA4
:1087B00002F05A6F4FEC02F05D6F4FEC02F05C6F0D
:1087C0004FEC02F05F6F4FEC02F05E6F4FEC02F087
:1087D000616F4FEC02F0606F4FEC02F0636F4FEC93
:1087E00002F0626F4FEC02F0656F4DEC02F0646FC7
:1087F0007EEC02F0A1EC02F0EE0E6BEC02F0B60E95
:108800006BEC02F04FEC02F0676F4FEC02F0666F1A
:108810004FEC02F0696F4FEC02F0686F4FEC02F022
:10882000816F4FEC02F0806F4FEC02F0836F4FECE2
:1088300002F0826F4FEC02F0856F4DEC02F0846F16
:108840007EEC02F0718E00011200719E8BD8A9C3DC
:1088500089F3A8C388F3A7C387F3A6C386F3A5C388
:108860008DF3A4C38CF3A3C38BF3A2C38AF3C80E06
:1088700033EC03F077D8A9C395F3A8C394F3A7C347
:1088800093F3A6C392F3A5C399F3A4C398F3A3C328
:1088900097F3A2C396F3C80E33EC03F063D8030139
:1088A0008651A625236E8751A721246E8851A821C1
:1088B000256E8951A921266E92512324866F9351EA
:1088C0002420876F94512520886F95512620896F29
:1088D00089C313F088C312F087C311F086C310F068
:1088E0001B6A1A6A196A030E186ED3EC03F013C0E0
:1088F000A9F312C0A8F311C0A7F310C0A6F39651B4
:108900008A25236E97518B21246E98518C21256ED8
:1089100099518D21266EA25123248A6FA3512420C0
:108920008B6FA45125208C6FA55126208D6F8DC390
:1089300013F08CC312F08BC311F08AC310F01B6AC2
:108940001A6A196A030E186ED3EC03F013C0A5F36C
:1089500012C0A4F311C0A3F310C0A2F3000148D8C1
:10896000718E1200A1EC02F0EE0E6BEC02F0F40E30
:108970006BEC02F02E0E69EC02F0050E33EC03F006
:10898000EE0E6BEC02F0F60E6BEC02F04FEC02F028
:108990000301B36F4DEC02F0B26F7EEC02F0B3C393
:1089A000A3F3B2C3A2F3A1EC02F0EE0E6BEC02F063
:1089B000F40E6BEC02F0340E69EC02F0050E33ECB1
:1089C00003F0EE0E6BEC02F0F60E6BEC02F04FECE7
:1089D00002F0B46F4FEC02F0B36F4DEC02F0B26FE7
:1089E0007EEC02F0B4C3A7F3B3C3A6F300011200F8
:1089F00003016451A25D316E6551A359326E000EC0
:108A000065BFFF0EA459336E000E65BFFF0EA5595A
:108A1000346E41EC08F034C026F033C025F032C08B
:108A200024F031C023F063C332F062C331F035EC7F
:108A300008F026C038F025C037F024C036F023C037
:108A400035F094EC07F034C024F333C023F332C084
:108A500022F331C021F324C3BDF323C3BCF322C3EB
:108A6000BBF30F0E215D02E23D84000E0301BA6FDD
:108A700083C332F082C331F035EC08F034C026F005
:108A800033C025F032C024F031C023F00B0E232474
:108A900002E33D82FF0E0001236EBDC32AF0BCC37A
:108AA00029F0BBC328F0BAC327F085C332F084C3D2
:108AB00031F035EC08F02AC038F029C037F028C072
:108AC00036F027C035F0A0EC06F034C02AF033C0F1
:108AD00029F032C028F031C027F026C034F025C07C
:108AE00033F024C032F023C031F02AC038F029C05E
:108AF00037F028C036F027C035F02EEC07F034C030
:108B0000C1F333C0C0F332C0BFF331C0BEF3BDC345
:108B100038F0BCC337F0BBC336F0BAC335F0C1C3BD
:108B200034F0C0C333F0BFC332F0BEC331F0A0ECA9
:108B300006F034C0D1F333C0D0F332C0CFF331C02C
:108B4000CEF3346A336A326A820E316ED1C338F0A2
:108B5000D0C337F0CFC336F0CEC335F0A0EC06F06B
:108B600034C026F033C025F032C024F031C023F0E9
:108B7000386A376A366A830E356E26C034F025C0EF
:108B800033F024C032F023C031F02EEC07F0E2ECD9
:108B900007F00301AA6F32C0ABF333C0ACF334C0AB
:108BA000ADF3386A376A200E366E820E356EADC36D
:108BB00034F0ACC333F0ABC332F0AAC331F041ECB4
:108BC00008F02EEC07F034C011F433C010F432C0BA
:108BD0000FF431C00EF4386A376A7A0E366E8A0E98
:108BE000356ED1C334F0D0C333F0CFC332F0CEC32F
:108BF00031F09EEC06F034C0D5F333C0D4F332C06C
:108C0000D3F331C0D2F3D5C338F0D4C337F0D3C3D4
:108C100036F0D2C335F0D5C334F0D4C333F0D3C368
:108C200032F0D2C331F094EC07F034C026F033C0F8
:108C300025F032C024F031C023F026C024F325C033
:108C400023F324C022F30C0E235C02E23D84000EC9
:108C50000301216F69C332F068C331F035EC08F0CD
:108C600024C338F023C337F022C336F021C335F0D4
:108C700094EC07F034C0BDF333C0BCF332C0BBF397
:108C800031C0BAF35DC332F05CC331F035EC08F0AB
:108C9000D5C338F0D4C337F0D3C336F0D2C335F0E0
:108CA00094EC07F034C0C1F333C0C0F332C0BFF35B
:108CB00031C0BEF3BDC338F0BCC337F0BBC336F020
:108CC000BAC335F0C1C334F0C0C333F0BFC332F010
:108CD000BEC331F0A0EC06F034C026F033C025F05E
:108CE00032C024F031C023F026C0C5F325C0C4F340
:108CF00024C0C3F30B0E235C02E23D84000E03018B
:108D0000C26F5BC332F05AC331F035EC08F034C0A7
:108D100026F033C025F032C024F031C023F0020E1B
:108D2000232402E33D82FF0E0001236E26C038F0AB
:108D300025C037F024C036F023C035F0C5C334F069
:108D4000C4C333F0C3C332F0C2C331F0A0EC06F0A9
:108D500034C026F033C025F032C024F031C023F0F7
:108D6000346A336A326A800E316E26C038F025C00C
:108D700037F024C036F023C035F0A0EC06F034C044
:108D800026F033C025F032C024F031C023F026C0D5
:108D9000C9F325C0C8F324C0C7F3020E235C02E266
:108DA0003D84000E0301C66F5FC332F05EC331F035
:108DB00035EC08F0D5C338F0D4C337F0D3C336F060
:108DC000D2C335F094EC07F034C026F033C025F060
:108DD00032C024F031C023F026C0BDF325C0BCF35F
:108DE00024C0BBF30D0E235C02E23D84000E0301A0
:108DF000BA6F67C332F066C331F035EC08F024C3B4
:108E000038F023C337F022C336F021C335F094EC99
:108E100007F034C026F033C025F032C024F031C052
:108E200023F026C0C1F325C0C0F324C0BFF3100E49
:108E3000235C02E23D84000E0301BE6FBDC326F039
:108E4000BCC325F0BBC324F0BAC323F026C038F05E
:108E500025C037F024C036F023C035F0C1C334F04C
:108E6000C0C333F0BFC332F0BEC331F0A0EC06F094
:108E700034C026F033C025F032C024F031C023F0D6
:108E8000346A336A326A800E316E26C038F025C0EB
:108E900037F024C036F023C035F0A0EC06F034C023
:108EA00026F033C025F032C024F031C023F026C0B4
:108EB000C5F325C0C4F324C0C3F3020E235C02E251
:108EC0003D84000E0301C26F61C332F060C331F014
:108ED0003DEC08F034C026F033C025F032C024F059
:108EE00031C023F0C5C32AF0C4C329F0C3C328F09E
:108EF000C2C327F0346A336A326A8E0E316E2AC0DA
:108F000038F029C037F028C036F027C035F0A0EC83
:108F100006F034C02AF033C029F032C028F031C046
:108F200027F026C038F025C037F024C036F023C023
:108F300035F02AC034F029C033F028C032F027C001
:108F400031F094EC07F034C026F033C025F032C085
:108F500024F031C023F026C0CDF325C0CCF324C0CB
:108F6000CBF30F0E235C02E23D84000E0301CA6FB7
:108F7000A9C334F0A8C333F0A7C332F0A6C331F0BD
:108F800041EC08F0C9C338F0C8C337F0C7C336F0A6
:108F9000C6C335F09EEC06F034C026F033C025F091
:108FA00032C024F031C023F0346A500E336E430EC9
:108FB000326E8E0E316E26C038F025C037F024C0D8
:108FC00036F023C035F094EC07F0E2EC07F07A6F4E
:108FD00032C07BF333C07CF334C07DF37DC334F007
:108FE0007CC333F07BC332F07AC331F041EC08F03C
:108FF000386A376A366A800E356E94EC07F034C0F2
:1090000026F033C025F032C024F031C023F026C052
:1090100034F025C033F024C032F023C031F0CDC38A
:1090200038F0CCC337F0CBC336F0CAC335F02EECE2
:1090300007F034C0D9F333C0D8F332C0D7F331C00E
:10904000D6F3D9C324F3D8C323F3D7C322F3080E2E
:10905000D65D02E23D84000E0301216F24C338F087
:1090600023C337F022C336F021C335F024C334F0D4
:1090700023C333F022C332F021C331F094EC07F064
:1090800034C0BDF333C0BCF332C0BBF331C0BAF35C
:10909000346AE00E336E3D0E326E8A0E316EBDC301
:1090A00038F0BCC337F0BBC336F0BAC335F094EC2C
:1090B00007F034C026F033C025F032C024F031C0B0
:1090C00023F026C0BDF325C0BCF324C0BBF3100EB3
:1090D000235C02E23D84000E0301BA6F346AE80E9D
:1090E000336EE50E326E8B0E316ED9C338F0D8C3B5
:1090F00037F0D7C336F0D6C335F094EC07F034C060
:1091000026F033C025F032C024F031C023F026C051
:10911000C1F325C0C0F324C0BFF3100E235C02E2EC
:109120003D84000E0301BE6FD9C326F0D8C325F0DD
:10913000D7C324F0D6C323F0BDC32AF0BCC329F0A3
:10914000BBC328F0BAC327F02AC038F029C037F0D3
:1091500028C036F027C035F0C1C334F0C0C333F0A7
:10916000BFC332F0BEC331F0A0EC06F034C02AF029
:1091700033C029F032C028F031C027F0346AF00E35
:10918000336E6C0E326E8A0E316E2AC038F029C0F2
:1091900037F028C036F027C035F0A0EC06F034C018
:1091A0002AF033C029F032C028F031C027F0040E75
:1091B000275E02E23D84276A000126C038F025C000
:1091C00037F024C036F023C035F02AC034F029C06F
:1091D00033F028C032F027C031F0A0EC06F0E2EC0A
:1091E00007F00301AE6F32C0AFF333C0B0F334C049
:1091F000B1F3386A376A480E366E850E356EB1C3E4
:1092000034F0B0C333F0AFC332F0AEC331F041EC51
:1092100008F02EEC07F034C026F033C025F032C041
:1092200024F031C023F09A0E346E990E336E4D0E39
:10923000326E830E316E26C038F025C037F024C060
:1092400036F023C035F0A0EC06F034C0D9F333C0BB
:10925000D8F332C0D7F331C0D6F300011200B50EF7
:109260000201896F620E8A6F060E8B6F240E8C6F5F
:109270008D6F8E6B8F699069060E916F030E926FE2
:10928000936B946B956B966B100E976F270E986F80
:10929000996B9A6B050E9B6F9C6BFA0E9D6F9E6B84
:1092A0009F6FA06B640EA16FA26B2C0EA36F010EBB
:1092B000A46FA56BA66BA76BA86BA96BAA6BAB6B16
:1092C000AC6BAD6BAE6BAF6BB06BB16BB26B160EC4
:1092D000B36FDC0EB46FB36BB46B020EC06F2A0EAB
:1092E0000201C05D000118E20201B3510E6E02EEF0
:1092F00089F0C051EB500F6E0E240C6E0CC0B3F20F
:10930000B4510E6EB3510F6E0E240C6E0CC0B4F23D
:109310000201C02B0001E3E30201C06B2C0E02012D
:10932000C05D000116E2800E026E400E096E216AD9
:1093300040C320F0066A056A200E016E02EE89F035
:109340000201C051EB50B3EC01F00201C02B00014F
:10935000E5E38BC20CF00CC08FF28CC20CF00CC099
:1093600090F2B50E0201896F620E8A6F050E8B6F47
:10937000010E8C6F020E8D6F8E6B916B926B020ED5
:10938000C06F080E0201C05D000118E20201915198
:109390000E6E02EE89F0C051EB500F6E0E240C6E73
:1093A0000CC091F292510E6E91510F6E0E240C6E04
:1093B0000CC092F20201C02B0001E3E3800E026EAA
:1093C000800E096E216A40C320F00B0E066EB80EA7
:1093D000056E72EC01F0D8A047D003011C6F0201AA
:1093E00089510C6E03011C510C5C000112E0800ECF
:1093F000026E800E096E216A40C320F00B0E066ECD
:10940000B80E056E72EC01F02FE303011C6F000132
:10941000E6D7010E0201C06F080E0201C05D000117
:109420001FE2800E026E800E096E216A40C320F09A
:109430000B0E066EB80E056E72EC01F015E303011B
:109440001C6F02EE89F00201C051EB500C6E03015B
:109450001C510C5C000108E10201C02B0001DCE39F
:1094600003012A950001120003012A850001120060
:089470000400FED70400FED742
:020000040030CA
:03000100C80E33F3
:020005003D803C
:0600080008C00FE00F40EC
:0200000400F00A
:100000004243303553FFFFFFFFFFFFFFFFFFFFFFBE
:100010004243504C35FFFFFFFFFFFFFFFFFF34332C
:1000200034393235303030FFFFFFFFFFFFFF383506
:1000300030FFFFFFFFFFFFFFFFFFFFFFFFFF31303C
:1000400030FFFFFFFFFFFFFFFFFFFFFFFFFF373224
:10005000FFFFFFFFFFFFFFFFFFFFFFFFFFFF353049
:10006000FFFFFFFFFFFFFFFFFFFFFFFFFFFF32303C
:10007000FFFFFFFFFFFFFFFFFFFFFFFFFFFF69091C
:100080000606F82401B004544400FFFFFFFF6A296C
:100090003F3E3C3830202123272F475501310611A0
:1000A000150902140B10041E0D1207050F161B0A6A
:0800B00008030C180E191D13C2
:00000001FF
